:020000020000FC
:100000000C94353B189518951895189518951895D2
:100010001895189518951895189518951895189578
:100020001895189518951895189518951895189568
:100030001895189518951895189518951895189558
:100040001895189518951895189518951895189548
:100050000C94961418951895189518951895189548
:100060001895189518951895189518951895189528
:100070001895189518951895189518951895189518
:100080001895189518951895189518951895189508
:1000900018951895189518951895189518951895F8
:1000A00018951895189518951895189518951895E8
:1000B00018951895189518951895189518951895D8
:1000C00018951895189518951895189518951895C8
:1000D00018951895189518951895189518951895B8
:1000E00018951895189518951895189518951895A8
:1000F0001895189518951895189518951895189598
:100100001895189518951895189518951895189587
:100110001895189518951895189518950C94891494
:100120001895189518951895189518951895189567
:10013000189518950C9411141895189518951895EC
:100140001895189518951895189518951895189547
:100150001895189518951895189518951895189537
:100160001895189518951895189518951895189527
:100170001895189518951895189518951895189517
:100180001895189518951895189518951895189507
:1001900018951895189518951895189518951895F7
:1001A00018951895189518951895189518951895E7
:1001B00018951895189518951895189518951895D7
:1001C00018951895189518951895189518951895C7
:1001D00018951895189518951895189518951895B7
:1001E00018951895189518951895189518951895A7
:1001F00018951895189518951895189500000000F1
:1002000000000000000000000000000000000000EE
:1002100000000000000000000000000000000000DE
:1002200000000000000000000000000000000000CE
:1002300000000000000000000000000000000000BE
:1002400000000000000000000000000000000000AE
:10025000000000000000000000000000000000009E
:10026000000000000000000000000000000000008E
:10027000000000000000000000000000000000007E
:10028000000000000000000000000000000000006E
:10029000000000000000000000000000000000005E
:1002A000000000000000000000000000000000004E
:1002B000000000000000000000000000000000003E
:1002C000000000000000000000000000000000002E
:1002D000000000000000000000000000000000001E
:1002E000000000000000000000000000000000000E
:1002F00000000000000000000000000000000000FE
:1003000000000000000000000000000000000000ED
:1003100000000000000000000000000000FFFFFFE0
:10032000FFFFFFFFFFFFFFFFFFFFFFFFFFFFFFFFDD
:1003300000000000000000000000000000000000BD
:1003400000000000000000000000000000000000AD
:10035000000000000000000000000000000000009D
:100360000000000000000000000000000080C0C08D
:10037000C08000000000000000000000000000003D
:1003800000000000070F1F3F3F1F0F060000000086
:10039000000000000000000000000000000000005D
:1003A000000000000000000000000000000000004D
:1003B00000000000387CFEFFFFFE7C3800000000DB
:1003C000000000000000000000000000000000012C
:1003D0000100000000000000000000000000C0E07C
:1003E000F0F8FCFCFCFCFCFCFCFCFCFCFCFCF8F06D
:1003F000E0C000000000FFFFFFFFFFFF0000000063
:1004000000000000FFFFFFFFFFFF00000000FFFFF4
:10041000FFFFFFFF0000000000000000FFFFFFFFE4
:10042000FFFF00000000FFFFFFFFFFFF00000000D4
:1004300000000000FFFFFFFFFFFF000000000307B8
:100440000F1F3F3F3F3F3F3F3F3F3F3F3F3F1F0F5C
:10045000070300000000C0E0F0F8FCFCFCFCFCFC22
:10046000FCFCFC0000000000000000000000000098
:100470000000000000FFFFFFFFFFFF000000000082
:1004800000000000000000000000000000FFFFFF6F
:10049000FFFFFF000000000000000000000000005F
:1004A0000000000000FFFFFFFFFFFF000000000052
:1004B000000000000000000000000000003F3F3F7F
:1004C0003F3F3F0000000000000000000000C0E0CF
:1004D000F0F8FCFCFCFCFCFCFCFCFCFCFCFCF8F07C
:1004E000E0C000000000000000000000000000006C
:1004F00000000000FFFFFFFFFFFF00000000C0E062
:10050000F0F8FCFE7E7E7E7E7E7E7E7E7F3F1F0F2D
:10051000070300000000FFFFFFFFFFFF00000000D7
:1005200000000000000000000000000000000307C1
:100530000F1F3F3F3F3F3F3F3F3F3F3F3F3F3E3C1F
:100540003830000000000C1C3C7CFCFCFCFCFCFC7B
:10055000FCFCFCFCFCFCF8F0E0C00000000000002B
:10056000000000000000000000000000FFFFFFFF8F
:10057000FFFF00000000000000007E7E7E7E7E7E89
:100580007E7E7E7EFFFFFFFFE7C3000000000000CD
:10059000000000000000000000000000FFFFFFFF5F
:1005A000FFFF0000000030383C3E3F3F3F3F3F3FF1
:1005B0003F3F3F3F3F3F1F0F070300000000FCFC91
:1005C000F8F0E0C00000000000000000C0E0F0F81B
:1005D000FCFC00000000FFFFFFFFFFFF0000000029
:1005E00000000000FFFFFFFFFFFF00000000070FFB
:1005F0001F3F7F7F7E7E7E7E7E7E7E7EFFFFFFFFB3
:10060000FFFF0000000000000000000000000000EC
:1006100000000000FFFFFFFFFFFF000000000000E0
:1006200000000000000000000000000003070F1F92
:100630003F3F00000000C0E0F0F8FCFCFCFCFCFCCC
:10064000FCFCFCFCFCFC7C3C1C0C00000000FFFFE4
:10065000FFFFFFFF0000000000000000000000009E
:10066000000000000000070F1F3F7F7F7E7E7E7E20
:100670007E7E7E7EFEFEFCF8F0E0000000000000C2
:10068000000000000000000000000000FFFFFFFF6E
:10069000FFFF0000000003070F1F3F3F3F3F3F3FAA
:1006A0003F3F3F3F3F3F1F0F070300000000C0E0F8
:1006B000F0F8FCFCFCFCFCFCFCFCFCFCFCFC7C3CCA
:1006C0001C0C00000000FFFFFFFFFFFF0000000008
:1006D0000000000000000000000000000000FFFF1C
:1006E000FFFFFFFF7E7E7E7E7E7E7E7EFEFEFCF82E
:1006F000F0E000000000FFFFFFFFFFFF0000000030
:1007000000000000FFFFFFFFFFFF000000000307E5
:100710000F1F3F3F3F3F3F3F3F3F3F3F3F3F1F0F89
:100720000703000000000C1C3C7CFCFCFCFCFCFCF7
:10073000FCFCFCFCFCFCF8F0E0C000000000000049
:10074000000000000000000000000000FFFFFFFFAD
:10075000FFFF00000000000000000000000000009B
:1007600000000000FFFFFFFFFFFF0000000000008F
:10077000000000000000000000000000FFFFFFFF7D
:10078000FFFF00000000000000000000000000006B
:100790000000000003070F1F3F3F00000000C0E003
:1007A000F0F8FCFCFCFCFCFCFCFCFCFCFCFCF8F0A9
:1007B000E0C000000000FFFFFFFFFFFF000000009F
:1007C00000000000FFFFFFFFFFFF00000000C3E785
:1007D000FFFFFFFF7E7E7E7E7E7E7E7EFFFFFFFF31
:1007E000E7C300000000FFFFFFFFFFFF0000000065
:1007F00000000000FFFFFFFFFFFF000000000307F5
:100800000F1F3F3F3F3F3F3F3F3F3F3F3F3F1F0F98
:10081000070300000000C0E0F0F8FCFCFCFCFCFC5E
:10082000FCFCFCFCFCFCF8F0E0C000000000FFFF5A
:10083000FFFFFFFF0000000000000000FFFFFFFFC0
:10084000FFFF00000000070F1F3F7F7F7E7E7E7E40
:100850007E7E7E7EFFFFFFFFFFFF000000000000A6
:10086000000000000000000000000000FFFFFFFF8C
:10087000FFFF0000000030383C3E3F3F3F3F3F3F1E
:100880003F3F3F3F3F3F1F0F0703000000000000B6
:100890000000000000000000000000000000000058
:1008A0000000000000000000000000000000000048
:1008B0000000000000000000000000000000000038
:1008C0000000000000000000000000000000001018
:1008D0003838383838383838100000000000000048
:1008E0000000000000000000000000000000000008
:1008F00000000000000000000000000000000000F8
:1009000000000000000000000000000000000000E7
:1009100000000000000000000000000000000002D5
:10092000060E0E0E0E0E0E06020000000000001055
:100930003838383838383838100000000000008067
:10094000C0E0E0E0E0E0E0C0800000000000FCFA71
:10095000F60E0E0E0E0E0EF6FAFC00000000EFC7AB
:100960008300000000000083C7EF000000007FBF8D
:10097000DFE0E0E0E0E0E0DFBF7F0000000000003B
:1009800000000000000000F0F8FC00000000000083
:100990000000000000000083C7EF0000000000001E
:1009A000000000000000001F3F7F00000000000268
:1009B000060E0E0E0E0E0EF6FAFC00000000E0D041
:1009C000B83838383838383B170F000000007FBF80
:1009D000DFE0E0E0E0E0E0C08000000000000002B6
:1009E000060E0E0E0E0E0EF6FAFC000000000010B1
:1009F00038383838383838BBD7EF0000000000806E
:100A0000C0E0E0E0E0E0E0DFBF7F00000000FCF8D5
:100A1000F0000000000000F0F8FC000000000F17DC
:100A20003B383838383838BBD7EF000000000000BA
:100A3000000000000000001F3F7F00000000FCFAE3
:100A4000F60E0E0E0E0E0E060200000000000F172E
:100A50003B383838383838B8D0E000000000008023
:100A6000C0E0E0E0E0E0E0DFBF7F00000000FCFA73
:100A7000F60E0E0E0E0E0E06020000000000EFD75E
:100A8000BB383838383838B8D0E0000000007FBFB5
:100A9000DFE0E0E0E0E0E0DFBF7F00000000000218
:100AA000060E0E0E0E0E0EF6FAFC00000000000000
:100AB0000000000000000083C7EF000000000000FD
:100AC000000000000000001F3F7F00000000FCFA53
:100AD000F60E0E0E0E0E0EF6FAFC00000000EFD71A
:100AE000BB383838383838BBD7EF000000007FBF3C
:100AF000DFE0E0E0E0E0E0DFBF7F00000000FCFAC4
:100B0000F60E0E0E0E0E0EF6FAFC000000000F1789
:100B10003B383838383838BBD7EF00000000008049
:100B2000C0E0E0E0E0E0E0DFBF7F000000000000A8
:100B3000000000000000000000000000000038FC81
:100B4000FC3800000000000D0D000000000E1E002B
:100B5000001E0E00000000000000000020F8F82039
:100B6000F8F82000020F0F020F0F0200387C4447F4
:100B700047CC9800060C0838380F0700303000804A
:100B8000C06030000C060301000C0C0080D87CE42F
:100B9000BCD84000070F0808070F080000101E0E01
:100BA0000000000000000000000000000000F0F85D
:100BB0000C040000000003070C0800000000040CF7
:100BC000F8F000000000080C0703000080A0E0C05F
:100BD000C0E0A0800002030101030200008080E069
:100BE000E08080000000000303000000000000001F
:100BF000000000000000101E0E00000080808080B9
:100C00008080800000000000000000000000000064
:100C1000000000000000000C0C000000000000803C
:100C2000C06030000C06030100000000F8F80CC49E
:100C30000CF8F00003070C080C070300001018FC68
:100C4000FC0000000008080F0F080800080C84C40E
:100C5000643C18000E0F0908080C0C00080C4444F2
:100C600044FCB800040C0808080F0700C0E0B09866
:100C7000FCFC8000000000080F0F08007C7C44444E
:100C800044C48400040C0808080F0700F0F84C4422
:100C900044C08000070F0808080F07000C0C0484EC
:100CA000C47C3C0000000F0F00000000B8FC44446E
:100CB00044FCB800070F0808080F0700387C4444BC
:100CC00044FCF800000808080C070300000000308E
:100CD00030000000000000060600000000000030A8
:100CE000300000000000080E060000000080C06018
:100CF0003018080000000103060C08000020202026
:100D0000202020000001010101010100000818302D
:100D100060C0800000080C0603010000181C04C419
:100D2000E43C18000000000D0D000000F0F008C8C1
:100D3000C8F8F000070F080B0B0B0100E0F0988CCF
:100D400098F0E0000F0F0000000F0F0004FCFC44BF
:100D500044FCB800080F0F08080F0700F0F80C0457
:100D6000040C180003070C08080C060004FCFC0423
:100D70000CF8F000080F0F080C07030004FCFC44FB
:100D8000E40C1C00080F0F08080C0E0004FCFC44C7
:100D9000E40C1C00080F0F0800000000F0F80C84A1
:100DA000848C980003070C0808070F00FCFC4040E7
:100DB00040FCFC000F0F0000000F0F00000004FCBF
:100DC000FC0400000000080F0F08000000000004F1
:100DD000FCFC0400070F08080F07000004FCFCC01F
:100DE000E03C1C00080F0F00010F0E0004FCFC0487
:100DF00000000000080F0F08080C0E00FCFC387003
:100E000038FCFC000F0F0000000F0F00FCFC3870D6
:100E1000E0FCFC000F0F0000000F0F00F8FC0404C2
:100E200004FCF800070F0808080F070004FCFC4446
:100E3000447C3800080F0F0800000000F8FC040490
:100E400004FCF800070F080E3C3F270004FCFC449C
:100E5000C4FC3800080F0F00000F0F00183C64445A
:100E6000C49C1800060E0808080F0700001C0CFCA4
:100E7000FC0C1C000000080F0F080000FCFC000028
:100E800000FCFC00070F0808080F0700FCFC00002E
:100E900000FCFC000103060C06030100FCFC000042
:100EA00000FCFC00070F0E030E0F07000C3CF0E0E7
:100EB000F03C0C000C0F0301030F0C00000C7CC075
:100EC000C07C3C000000080F0F0800001C0C84C40C
:100ED000643C1C000E0F0908080C0E000000FCFC0E
:100EE0000404000000000F0F080800003870E0C084
:100EF000800000000000000103070E000000040451
:100F0000FCFC0000000008080F0F0000080C06039E
:100F1000060C0800000000000000000000000000B7
:100F200000000000202020202020202000000307B7
:100F300004000000000000000000000000A0A0A0CD
:100F4000E0C00000070F0808070F080004FCFC20A1
:100F500060C08000000F0F08080F0700C0E02020CD
:100F600020604000070F0808080C040080C06024BF
:100F7000FCFC0000070F0808070F0800C0E0A0A055
:100F8000A0E0C000070F0808080C040040F8FC446B
:100F90000C180000080F0F0800000000C0E020201F
:100FA000C0E02000276F48487F3F000004FCFC4061
:100FB00020E0C000080F0F00000F0F00000020EC21
:100FC000EC0000000000080F0F0800000000000007
:100FD00020ECEC0000307040407F3F0004FCFC80BF
:100FE000C0602000080F0F01030E0C00000004FC7D
:100FF000FC0000000000080F0F080000E0E060C0E7
:1010000060E0C0000F0F0007000F0F0020E0C020BD
:1010100020E0C000000F0F00000F0F00C0E02020F4
:1010200020E0C000070F0808080F070020E0C020DC
:1010300020E0C000407F7F48080F0700C0E020206C
:10104000C0E02000070F08487F7F400020E0C0601C
:1010500020E0C000080F0F080000000040E0A020C2
:1010600020604000040C09090B0E04002020F8FC4D
:10107000202000000000070F080C0400E0E0000042
:10108000E0E00000070F0808070F080000E0E0009C
:1010900000E0E0000003070C0C070300E0E0008024
:1010A00000E0E000070F0C070C0F07002060C08075
:1010B000C0602000080C0703070C0800E0E00000F7
:1010C00000E0E000474F4848683F1F00606020A0F4
:1010D000E06020000C0E0B09080C0C00004040F8EA
:1010E000BC040400000000070F080800000000BC5A
:1010F000BC0000000000000F0F000000000404BC52
:10110000F84040000008080F07000000080C040C1D
:10111000080C04000000000000000000E0F0988CC3
:1011200098F0E0000F0F0000000F0F0004FCFC44DB
:1011300044CC8C00080F0F08080F070004FCFC4487
:1011400044FCB800080F0F08080F070004FCFC045B
:10115000040C0C00080F0F080000000000F8FC0C45
:10116000FCF800001C0F0F080F0F1C0004FCFC44CF
:10117000E40C1C00080F0F08080C0E000C3CE0FCEF
:10118000E03C0C000C0F010F010F0C00080C444454
:1011900044FCB800040C0808080F0700FCFC80C0E1
:1011A00060FCFC000F0F0100000F0F00FCFC80C270
:1011B00060FCFC000F0F0100000F0F0004FCFCC0DE
:1011C000E03C1C00080F0F00010F0E0000F0F81C9F
:1011D0000CFCFC00080F0F00000F0F00FCFC387027
:1011E00038FCFC000F0F0000000F0F00FCFC40401B
:1011F00040FCFC000F0F0000000F0F00F8FC04047F
:1012000004FCF800070F0808080F0700FCFC0404A2
:1012100004FCFC000F0F0000000F0F0004FCFC4456
:10122000447C3800080F0F0800000000F0F80C04A0
:10123000040C180003070C08080C0600001C0CFC2A
:10124000FC0C1C000000080F0F0800001C3C60C0D4
:1012500080FCFC0000000C0D07030100F0F808FC06
:1012600008F8F0000103020F020301000C3CF0E05B
:10127000F03C0C000C0F0301030F0C00FCFC000001
:10128000FCFC00000F0F08080F1F1800387CC080FE
:1012900080FCFC0000000000000F0F00FC00FCFCC4
:1012A00000FC00000F080F0F080F0000FC00FCFC02
:1012B00000FC00000F080F0F081F180004FCFC4082
:1012C00040C0C000080F0F08080C0F00FCFC40C015
:1012D000C000FC000F0F080C0F000F0000FCFC40CA
:1012E00040C0C000000F0F08080C0F000C0404C41D
:1012F000CCF8F0000C0808080C070300FCFC80F890
:101300000404F8000F0F0007080807000078CC84D9
:1013100084FCFC00080C0603010F0F0000A0A0A035
:10132000E0C00000070F0808070F0800E0E02020D9
:10133000202000000F0F090909060000E0E0A0A02E
:10134000A04000000F0F080808070000E0E0202080
:10135000206000000F0F00000000000000E02020CF
:10136000E00000001C0F0C0C0F1C0000C0E0A0A04F
:10137000A0E0C000070F0808080C040020E080E08F
:1013800080E02000080F010F010F0800402020A07E
:10139000E06000000408090906060000E0E0000023
:1013A00080E000000F0F0201000F0000E0E00010DD
:1013B00080E000000F0F0201000F000004FCFC8021
:1013C000C0602000080F0F01030E0C0000E0202079
:1013D000E0E00000080700000F0F0000E0C0000080
:1013E000C0E000000F000101000F0000E0E000007D
:1013F000E0E000000F0F01010F0F0000C0E020200F
:1014000020E0C000070F0808080F0700E0E02020D8
:10141000E0E000000F0F00000F0F000020E0C020F0
:1014200020E0C000407F7F48080F0700C0E0202078
:1014300020604000070F0808080C04002020E0E0AE
:101440002020000000000F0F0000000060C080009E
:10145000E0E000000C0C070301000000C020F0F0E9
:1014600020C0000003040F0F040300002060C080B0
:10147000C0602000080C0703070C0800E0E0000033
:1014800000E000000F0F0808080F1800E0E000005F
:10149000E0E00000010302020F0F0000E000E0E0C6
:1014A00000E000000F080F0F080F0000E000E0E070
:1014B00000E000000F080F0F081F100000000000E0
:1014C000000000000000000000000000E08080003C
:1014D00000E000000F080807000F000080808080F7
:1014E00080808000000000000000000040202020DC
:1014F000E0C00000040808090F070000E000C02059
:1015000020C000000F01070808070000C0202020AD
:10151000E0E00000080503010F0F000000000000DC
:1015200000000000000000000000000000000000BB
:101530000000002F00000007000700147F147F1434
:10154000242A7F2A12231308646236495522500048
:1015500005030000001C2241000041221C00140869
:101560003E081408083E08080000A06000080808AB
:101570000808006060000020100804023E51494540
:101580003E00427F400042615149462141454B3176
:101590001814127F1027454545393C4A4949300106
:1015A000710905033649494936064949291E00365D
:1015B00036000000563600000814224100141414AE
:1015C00014140041221408020151090632495951EC
:1015D0003E7C1211127C7F494949363E41414122ED
:1015E0007F4141221C7F494949417F090909013E48
:1015F0004149497A7F0808087F00417F4100204027
:10160000413F017F081422417F404040407F020C4F
:10161000027F7F0408107F3E4141413E7F09090956
:10162000063E4151215E7F09192946464949493103
:1016300001017F01013F4040403F1F2040201F3FEC
:101640004038403F6314081463070870080761516D
:10165000494543007F4141000106083040004141B7
:101660007F000402010204404040404000030500A6
:101670000020545454787F4844443838444444202B
:10168000384444487F3854545418087E09010218DD
:10169000A4A4A47C7F0804047800447D400040801A
:1016A000847D007F1028440000417F40007C0418A6
:1016B00004787C080404783844444438FC24242406
:1016C0001818242418FC7C08040408485454542096
:1016D000043F4440203C4040207C1C2040201C3CD7
:1016E0004030403C44281028441CA0A0A07C446406
:1016F000544C4400107C82000000FF000000827CFB
:10170000100008040810087C1211127C7F49494916
:10171000317F4545453A7F01010103603F213F602C
:101720007F49494941730C7F0C732141494D337FF7
:101730001008047F7E2011087E7F08142241403F5C
:1017400001017F7F0608067F7F0808087F3E414130
:10175000413E7F0101017F7F090909063E41414168
:101760002203017F010361261806011C227F221C2F
:1017700063140814633F20203F60070808087F7F38
:10178000407F407F3F203F207F017F4848307F4897
:1017900078007F7F484830004149492A1C7F103E2D
:1017A000413E661909097F20545478403E49454519
:1017B000387E4A4A34007C04040C00384545493ED2
:1017C00038545454184C307C304C24424A34007CF9
:1017D00020107C007C21117C007C10284400403CBF
:1017E00004047C7C0810087C7C10107C0038444485
:1017F00044387C04047C00FC1824241838444444F5
:101800002804047C04044C9090907C18247E2418B6
:1018100044281028443C20203C601C10107C007C94
:10182000407C407C3C203C207C047C5070007C5000
:1018300070007C7C50700000424252523C7C103858
:101840004438402C127E000000000000BFA731BECB
:101850007ED93BBE0F3AABBC82CB5B3EA166A73EB6
:1018600082CB5B3E0F3AABBC7ED93BBEBFA731BE3D
:101870000FBC5FBEBDF3E3BD5E5D2C3E0D13A53E08
:101880005E5D2C3EBDF3E3BD0FBC5FBE14BEA1BDCB
:101890006FEDFCBDDC252FBEE9383F3FDC252FBEB8
:1018A0006FEDFCBD14BEA1BD000102040824212C73
:1018B0002134213C2144214E2156215C21612169A2
:1018C00021702179218021882190219B21A721B19C
:1018D00021BD21C821D521DD21E421F021FB2107F3
:1018E0002213221A2220222C223822452251225D44
:1018F000226822742280228B229722A222AD22B754
:1019000022C222CD22D922E322EE22F82204230E83
:1019100023192323232E2338230102040A5A4723A1
:101920004B234E37A437B837C637D437F33706388A
:1019300014382538323850385E386C387A38913857
:10194000A038B338C238EA380C3929393A39503915
:10195000503950395039503950395039503950393F
:10196000503950395039503950395039503950392F
:10197000503950395039503950395039503950391F
:10198000503950395039503950395039503950390F
:1019900050395039503950395039503950395039FF
:1019A00050395039503950395039503950395039EF
:1019B00050395039503950395039503943397339C9
:1019C000B139BC39C739D039E739F039FA39053A74
:1019D000113A1C3A263A303A3B3A4A3A553A5F3A7B
:1019E0006A3A7F3A8E3A933A3A39503950395039F7
:1019F000503950395039503950395039503950399F
:101A0000503950395039503950395039503950398E
:101A1000503950395039503950395039503950397E
:101A2000503950395039503950395039503950396E
:101A3000503950395039503950395039503950395E
:101A4000503950395039503950395039503950394E
:101A500050395039503950399E3A0001E040DD404C
:101A600045D04002D040113A400BFF3F01584001A1
:101A7000D04001D04001D04002584005EC3F012D3C
:101A800040013A40030840023A40033640FB1BEC59
:101A90001093520018E010935000E1E5F0E010813F
:101AA00013FFFDCF00540483E0E500810061008353
:101AB000E1E5008104FFFDCF08ED04BF04E00093E1
:101AC0004000E0E500810E7F0083089501E000936F
:101AD000280200E300932902089501E000933002F8
:101AE00008E30093310208950DE00093200300E421
:101AF0000093210300E00093220300E400932403F9
:101B000000EE0093280300932A0300EE00932A03BB
:101B100008950895E4E6F6E010811E7F1083108199
:101B20001B7F108318E020812F7E208307FB2081FC
:101B300016F4286001C0277F208320812061208344
:101B4000000F1A9581F70895E4E6F6E010811E7FF4
:101B5000108310811460E5CFE4E6F6E000810E7F8B
:101B6000008300810D7F008304E610E0D2DFE4E60D
:101B7000F6E000810260008304E110E0CADF02EEBB
:101B8000C9DF0AE010E0C5DF0CE2C4DF0AE010E0C4
:101B9000C0DF0EE2BFDF04E110E0BBDF0FE2BADF1F
:101BA0000EE110E0B6DF0091480603FD02C005E239
:101BB00001C003E2AFDF01E8ADDF08E2ABDF02EA1C
:101BC000A9DF08ECA7DF00EAA5DF00E4A3DF0FEA46
:101BD000A1DFE4E6F6E000810160008308958A93C6
:101BE000812FE4E6F6E010811E7F10838A9501556F
:101BF00091DF082F02950F70005F8CDF8F70082F28
:101C000089DF89910895BA93AA939A938A93A02F12
:101C1000912FA05C88E0012F069506950695801B04
:101C20001A2F082FDCDF9770492F00E80E946A3BCB
:101C3000BA2FBB0FBB0B23E02B9F302D2A9F310DFA
:101C4000EAE0F7E2E00DF31F982F990F990BE80FE8
:101C5000F91F1081102B1083012F76DF0C940D1AC1
:101C6000392F482F8AE097E211E8FC0104E020E0D8
:101C700021930A95E9F703961A95B9F70FE30093B4
:101C8000CA2720939E2820939F282093A028209342
:101C9000A128842F932F08959A938A93E4E6F6E07F
:101CA00000810E7F008380E011E0082F039597DF0D
:101CB00094E800E049DF9A95E1F783958930A0F335
:101CC000E4E6F6E00081016000838991999108952E
:101CD000BA92AA929A928A927A926A925A924A9264
:101CE000BA93AA939A938A93B02FA12FC90144243F
:101CF000E4E6F6E000810E7F008322C05B2E0C52EA
:101D0000202F08E7029F2CEF622E21E0722E600C3C
:101D1000711C05E0A02E1A2F052D61DF430108E19B
:101D2000B02EF40105914F010FDFBA94D1F708E10D
:101D3000600E00E0701E5394AA9469F74394A85E65
:101D40005524FC01E40DF51D00810023B9F67FC088
:101D5000BA92AA929A928A927A926A925A924A92E3
:101D6000BA93AA939A938A93B02FA12FC9014424BE
:101D7000E4E6F6E000810E7F008323C05B2E0C5268
:101D8000202F08E7029F2CEF622E21E0722E600CBC
:101D9000711C05E0A02E1A2F052D21DF430108E15B
:101DA000B02EF40105914F010095CEDEBA94C9F72B
:101DB00008E1600E00E0701E5394AA9461F743940A
:101DC000A85E5524FC01E40DF51D00810023B1F649
:101DD0003EC0BA92AA929A928A927A926A925A9241
:101DE0004A92BA93AA939A938A93902F812FD901FA
:101DF0004424E4E6F6E000810E7F008321C0592EE2
:101E00000C5210E3019F0CE8602E08E0702E600C6D
:101E1000711C03E0A02E182F052DE1DE430100E127
:101E2000B02EF40105914F018FDEBA94D1F700E195
:101E3000600E00E0701E5394AA9469F74394805F8B
:101E40005524FD01E40DF51D00810023C1F68991A3
:101E50009991A991B99149905990699079908990F7
:101E60009990A990B9900895CA92BA92AA929A921A
:101E70008A927A926A925A924A92BA93AA939A93BF
:101E80008A93A02E912FD90180E00023F1F1E4E69E
:101E9000F6E000810E7F00830C91003818F400E218
:101EA000402E27C001E6FCCF5A2CFD01E80FF11FA0
:101EB0000081041910E1019F0CE2602E0BE0702EEE
:101EC000600C711C02E0B02E192F052D88DE430135
:101ED00008E0C02EF40105914F0136DECA94D1F717
:101EE00008E0600E00E0701E5394BA9469F7839581
:101EF000985F10E0FD01E80FF11F0081002329F039
:101F000000520F3D88F28395F4CF89919991A99160
:101F1000B991499059906990799089909990A99038
:101F2000B990C99008958A927A926A925A924A9286
:101F3000BA93AA939A938A93902F812FD90144241C
:101F4000E4E6F6E000810E7F00830C91003818F47F
:101F500000E2502E19C001E6FCCF602E6518182F44
:101F6000092F3DDE05E0609E0CE2602E05E1702E3B
:101F7000600C711C05E0802EF30105913F01E4DD4A
:101F80008A94D1F743948A5F10E0FD01E40DF11FBC
:101F90000081002311F789919991A991B9914990F4
:101FA000599069907990899008958A93812F102F84
:101FB000082F069506950695039511DE8770482F24
:101FC00001E00E94653BC0DD89910895AA939A9330
:101FD0008A93A02F812F98E0102F110F110B0E94D0
:101FE000C13A0F33104054F5A05C1A2F08E0F7DD1A
:101FF00000E0AADD1A2F07E0F2DD00E0A5DD1A2FD0
:1020000006E0EDDD00E0A0DD883030F01A2F08E0BA
:10201000E6DD0FEF99DD97E0803130F01A2F07E011
:10202000DEDD0FEF91DD96E01A2F092FD8DD8770E6
:10203000F0E0E82FE656F94D008186DD899199910F
:10204000A99108955A924A92BA93AA939A938A931D
:10205000B12F002309F448C080E0102F110F110B9D
:10206000065A1F4F4AE050E00E94B33B102F07E092
:10207000109F402C43945B2EB831D0F4052D07708F
:1020800009F480E086958058A42DA39597E01A2F37
:1020900008E0252D269526952695021BA0DD00E05B
:1020A00053DDA3959A9599F7539408E1501630F3B0
:1020B0005524BB23C9F0052D077009F480E08695EF
:1020C0008058A42DA39597E01A2F08E0252D26957A
:1020D00026952695021B83DD082F36DDA3959A955C
:1020E00099F753945B1638F30C94D1179A938A930B
:1020F000E4E6F6E000810E7F008386E011E0082F21
:102100006EDD94E800E020DD9A95E1F78395893053
:10211000A8F3D6CD8A93802F0A3008F089E0182FD3
:10212000110F1A5F2AE0281B06EF209F002D8ADF7F
:10213000182F110F1A5F0AE0081B29E0029F002DDB
:1021400081DF899108959A938A93902F80E0182FC8
:10215000165A04E044DD0FEFF7DC83959817B8F7C3
:102160008991999108958A9380E0182F165A04E076
:1021700036DD00E0E9DC83958E32B8F3899108956D
:1021800000392AE838E212E010F003E001C001E073
:102190006BCE9A928A926A925A924A92BA93AA9370
:1021A0009A938A9380E090E0A0E0B0E048E0642E4B
:1021B00042EC58E2FA01349700801180228033808B
:1021C000FA0100821182228233826A944450504084
:1021D000662081F7E2EAF8E26CC09A928A926A92EB
:1021E0005A924A92BA93AA939A938A9380E090E083
:1021F000A0E0B0E048E0642E46EE58E2FA013497E1
:102200000080118022803380FA01008211822282B4
:1022100033826A9444505040662081F7E6ECF8E23D
:1022200048C09A928A926A925A924A92BA93AA9310
:102230009A938A9380E090E0A0E0B0E046E0642EBC
:1022400042E059E2FA013497008011802280338005
:10225000FA0100821182228233826A9444505040F3
:10226000662081F7EAEEF8E27BC09A928A926A923F
:102270005A924A92BA93AA939A938A9380E090E0F2
:10228000A0E0B0E046E0642E4EE159E2FA01349756
:102290000080118022803380FA0100821182228224
:1022A00033826A9444505040662081F7E6E0F9E2B8
:1022B00057C000831183228333830CE4402E08E14E
:1022C000502E4A01F20145915591659175912F016A
:1022D000F40101911191219131914F010E941C3D16
:1022E000AC01BD010E94BB3CC801D901639409E067
:1022F000601640F3082F89919991A991B99149905D
:10230000599069908990999008959A928A926A92C8
:102310005A924A92BA93AA939A938A9380E090E051
:10232000A0E0B0E046E0642E4AE359E2FA013497B7
:102330000080118022803380FA0100821182228283
:1023400033826A9444505040662081F7E2E2F9E219
:1023500000831183228333830CE8402E08E107C0F9
:10236000008311832283338300E7402E08E1502E3F
:102370004A01F20145915591659175912F01F40142
:1023800001911191219131914F010E941C3DAC01AD
:10239000BD010E94BB3CC801D901639407E06016EF
:1023A00040F3A8CF9A928A926A925A924A92BA932A
:1023B000AA939A938A9380E090E0A0E0B0E046E090
:1023C000642E46E559E2FA0134970080118022809C
:1023D0003380FA0100821182228233826A9444504F
:1023E0005040662081F7EEE3F9E2B2CFBA92AA92AA
:1023F0009A928A927A926A925A924A928A93842FF5
:10240000583029F44DEC442E4CEC542E0FC059306A
:1024100031F44FE8442E42EC542E45E707C05A30C1
:1024200041F44AE0442E47ED542E43E2642E4DE33E
:10243000742EA201B3010E941C3D48015901A20162
:10244000B30100E010E020E83FE30E94FF3C44E0DD
:10245000849FF001E65AF64D40815181628173817B
:102460000E941C3DA401B5010E94BB3C44E0849F36
:10247000F001E65AF64D00831183228333830E94D4
:10248000693C0E945C3C8991E6CC7A926A925A92AD
:102490004A92AA938A93842FA52F0E945C3C44E021
:1024A000849FF001E252F64D408151816281738137
:1024B0000E94FF3C280139010A2F10E020E030E0A3
:1024C0000E94673CA801B901820193010E94953DD9
:1024D00044E0849FF001E252F64D408151816281D7
:1024E00073810E94BB3C44E0849FF001E252F64DB0
:1024F00000831183228333838991A9910C94BF1A9D
:1025000020E02093800427E3F801258328E021833D
:1025100021E024830895BA93AA939A938A93D801C9
:10252000922F832F08E5EA2FF12F068304EF11E0A5
:102530000E946A20FD01978304EF11E00E946A2047
:10254000FD01878304EF11E00E946A2007E00093F9
:1025500083040C940D1A9A938A93C80100EA14E03C
:10256000CFDF30E820E000EA14E0D5DF0CE211E034
:102570000E946A2031E320E000EA14E0CCDF39EB6E
:1025800022E000EA14E0C7DF3BE420E100EA14E0C7
:10259000C2DF8C5490408C0120E030E00E94673C08
:1025A0004DEC5CEC6CE47DE30E94953D0E94693C3F
:1025B000302F21E000EA14E0AEDF08EB1BE00E94C0
:1025C0006A208991999108951CD008E30093CA016B
:1025D000EF93FF930F932F93EBECF1E008ED21E0E5
:1025E00004BF20832F910F91FF91EF910091C601BD
:1025F0004091C5010090C40130E0202F142F002D20
:1026000008950091CF0107FDFCCF08951091480077
:1026100001E0009348002091A0003091A2000091B9
:10262000A2000C7F04600093A2004FB77894E8E406
:10263000F0E00081016000835091CD01EF93FF93A2
:102640000F932F93EBECF1E008ED21E004BF208322
:102650002F910F91FF91EF9103E00093CD018895A9
:1026600010832093A0003093A2005093CD014FBF60
:1026700008950091CF0107FDFCCF0895FADF009186
:10268000CF0101FF11C006E30093CA01EF93FF934E
:102690000F932F93EBECF1E008ED21E004BF2083D2
:1026A0002F910F91FF91EF9108959A938A93C8010A
:1026B000E0DFFC01E05CF140B79738F41091652C45
:1026C00009E0109F800D911D11C0803901E0900735
:1026D00068F41091642C0DE1109F90014091652CDD
:1026E00007E5049F200D311D820F931F8093C001C9
:1026F000892F8F718093C10100E00093C20106E031
:102700000093CA01EF93FF930F932F93EBECF1E04B
:1027100008ED21E004BF20832F910F91FF91EF91ED
:102720000091C401899199910895AA939A938A93EB
:10273000C801A22FF801E05CF140B79738F410917E
:10274000652C09E0109F800D911D11C0003901E03A
:10275000900768F41091642C0DE1109F9001409156
:10276000652C07E5049F200D311D820F931F86DF26
:1027700003E30093CA018093C001892F8F71809376
:10278000C10100E00093C201A093C40100930609B7
:102790000093460805E30093CA0138DF03E0009385
:1027A000060901E00093460889919991A99108953D
:1027B000AA939A938A93C801A22FF801E05CF14092
:1027C000B79738F41091652C09E0109F800D911D8A
:1027D00011C0003901E0900768F41091642C0DE1FC
:1027E000109F90014091652C07E5049F200D311D3D
:1027F000820F931F43DF03E30093CA018093C0015C
:10280000892F8F718093C10100E00093C201A093D2
:10281000C40105E30093CA01F9DE89919991A99158
:102820000895FA93EA932A921A920A927A936A93F3
:102830005A934A933A932A931A930A932FB6E0E055
:10284000F2E000810460008300912E2C0395009338
:102850002E2C10912D2C011710F0E0932E2C0091AE
:102860002E2C0F9FF001EC56F54D00811181009345
:102870003A0310933B0300912E2C12E0019FF001CC
:10288000EC58F54D00811181009338031093390302
:102890000091322C002371F10091B42B1091B52BD3
:1028A000212F220F220B40912E2C54E0459FF00146
:1028B000EC5CF44D4081518162817381400F511F66
:1028C000621F721F4083518362837383E1ECFBE2DA
:1028D000008111810F5F1F4F008311832091C32B53
:1028E0003091C42B0217130728F000E00093322C1C
:1028F000008301832FBE0991199129913991499142
:10290000599169917991099019902990E991F991DA
:1029100018951A930A9300911002109111020093D6
:10292000B42B1093B52B099119911895BA92AA92CC
:102930009A928A927A926A925A924A92BA93AA93F5
:102940009A938A93FA93EA933A922A921A920A9263
:102950007A936A935A934A933A932A931A930A93CF
:10296000BFB60091322C002309F07FC200913B2CAE
:10297000002331F5442400912D2C002309F46DC06F
:10298000A4E3BBE284E79BE258E0442D0D911D9146
:102990002D913C91139779DD0E94693CFC010193D4
:1029A000119321933193CF0100E00D930D930D937B
:1029B0000D93439400912D2C401608F04EC0E4CFA7
:1029C00000913E2C0830442400912D2C002320F14E
:1029D00009F443C0A4E3BBE284E79BE250913E2CA0
:1029E000442D0D911D912D913C9113970E945C3CBB
:1029F000FDDC0E94693CFC0101931193219331930A
:102A0000CF0100E00D930D930D930D93439400912E
:102A10002D2C401610F5E2CF01F1A4E3BBE284E7D0
:102A20009BE250913E2C5395442D0D911D912D917B
:102A30003C9113972ADD0E94693CFC01019311939C
:102A400021933193CF0100E00D930D930D930D93DE
:102A5000439400912D2C401620F30FEF0093322C5D
:102A6000E0E2FCE2008111810F5F1F4F00831183C0
:102A70000037174131F400E00083018301E0009347
:102A80004D2C00E0E3EDFBE200830183028303832E
:102A9000EFECFBE20083018302830383ECE5FCE2BD
:102AA000008301830283038300912D2C002309F40A
:102AB00078C0A4E7BBE204EB802E0AE2902E84EFFC
:102AC0009AE2A0902D2C0D911D912D913C91139780
:102AD0000E945C3C280139010D911D912D913C9182
:102AE00013970E945C3CA201B3010E941C3DECE5DF
:102AF000FCE240815181628173810E94BB3CECE524
:102B0000FCE20083118322833383EFECFBE200813C
:102B10001181228133810E945C3C280139010D9191
:102B20001D912D913C9113970E945C3CF4014191C1
:102B30005191619171914F010E941C3DA201B3011D
:102B40000E94BB3C0E94693CEFECFBE200831183D6
:102B500022833383E3EDFBE2008111812281338103
:102B60000E945C3C280139010D911D912D913D91F0
:102B70000E945C3CFC014191519161917191CF01A6
:102B80000E941C3DA201B3010E94BB3C0E94693C13
:102B9000E3EDFBE20083118322833383AA9409F0DF
:102BA00092CF00912D2C10E020E030E00E94673C95
:102BB000A801B901ECE5FCE2008111812281338199
:102BC0000E94953D0E940043ECE5FCE200831183E6
:102BD000228333830091C72B1091C82B20E030E073
:102BE0000E94673CA801B901ECE5008111812281B6
:102BF00033810E94953D0E94693CE091402CF0E0B9
:102C0000E855F74E449150E00E949B3B0093BF2B48
:102C10001093C02BEFECFBE2008111812281338104
:102C2000EFEDFBE20083118322833383E3EDFBE2CC
:102C30000081118122813381E3EEFBE20083118365
:102C400022833383EBEEFBE2008111812281338109
:102C5000EFEDFBE24081518162817381041715071A
:102C600026073707EBEEFBE22CF40F5F1F4F2F4FC9
:102C70003F4F04C00150104020403040008311837A
:102C800022833383E7EEFBE20081118122813381CD
:102C9000E3EEFBE2408151816281738104171507E5
:102CA00026073707E7EEFBE22CF40F5F1F4F2F4F8D
:102CB0003F4F04C00150104020403040008311833A
:102CC000228333830091312C0023A9F000E000938C
:102CD000312CEFEDFBE20081118122813381EBEE9B
:102CE000FBE20083118322833383E7EEFBE2408320
:102CF000518362837383EBEEFBE2008111812281B9
:102D00003381EFEDFBE24081518162817381401B91
:102D1000510B620B730B4083518362837383E7EE25
:102D2000FBE20081118122813381E3EEFBE24081ED
:102D3000518162817381401B510B620B730B408385
:102D4000518362837383EFEDFBE200811181228165
:102D50003381E7E0FCE20083118322833383EBE0DD
:102D6000FCE2408351836283738300913B2C0130EA
:102D700009F055C00091492C0130F9F40091DF2B86
:102D80000E945C3C06DA0E94693CEFEFFBE20083A4
:102D9000118322833383E3EEFBE2008111812281E0
:102DA00033810E945C3C19DA0E94693CE3E0FCE25A
:102DB000008311832283338340C00230B9F4009131
:102DC000DF2B0E945C3C2DDA0E94693CEFEFFBE2B6
:102DD0000083118322833383E3EEFBE200811181C0
:102DE000228133810E945C3C40DADECF033029F53A
:102DF0000091DF2B0E945C3C88DA0E94693CEFEF77
:102E0000FBE20083118322833383E3EEFBE2008144
:102E10001181228133810E945C3CC4DAC5CF0091CC
:102E2000DF2BEFEFFBE20083118322833383E3E0A8
:102E3000FCE24083518362837383EFEFFBE2008106
:102E4000118122813381E7EDFBE20083118322832C
:102E50003383E3E0FCE20081118122813381EBEDD9
:102E6000FBE2008311832283338301E00093452C2E
:102E7000BFBE09911991299139914991599169914F
:102E800079910990199029903990E991F991899156
:102E90009991A991B99149905990699079908990A7
:102EA0009990A990B99018955A924A92BA93AA9378
:102EB0009A938A93280180E090E000912D2C0023C2
:102EC00089F1A4EBBAE240912D2C50E008E611E024
:102ED0000E94B33B189F102D099F100D089F002DD5
:102EE000110D040D151D083621E0120714F00856C7
:102EF0001140212F220F220B322F0E945C3C45E310
:102F00005AEF6EE87CE30E941C3D0E9432420D9312
:102F10001D932D933D93019600912D2C10E0801769
:102F200091078CF23EC05A924A92BA93AA939A930E
:102F30008A93280180E090E000912D2C002389F1F4
:102F4000A4EFBAE240912D2C50E008E611E00E9477
:102F5000B33B189F102D099F100D089F002D110DD8
:102F6000040D151D083621E0120714F00856114013
:102F7000212F220F220B322F0E945C3C45E35AEF97
:102F80006EE87CE30E941C3D0E94313B0D931D9333
:102F90002D933D93019600912D2C10E08017910701
:102FA0008CF289919991A991B9914990599008957C
:102FB000DA92CA92BA92AA929A928A927A926A9271
:102FC0005A924A92BA93AA939A938A93680180E09C
:102FD00090E000912D2C002309F446C0A4E9BAE248
:102FE00086012D2D220F220B322F0E945C3C4801BE
:102FF000590100912D2C10E020E030E00E94673C48
:10300000A801B9010BED1FE029EC30E40E94953DC9
:10301000280139018C01292F220F220B322F0E9407
:103020005C3CA201B3010E941C3D0E943242A401FB
:10303000B5010E941C3D2801390186012D2D220F6A
:10304000220B322F0E945C3CA201B3010E94BB3CC8
:103050000E94693C0D931D93019600912D2C10E068
:10306000801791070CF4BCCF89919991A991B991DE
:10307000499059906990799089909990A990B990C8
:10308000C990D9900895BA92AA929A928A927A9205
:103090006A925A924A92BA93AA939A938A9358013F
:1030A00049016624772400912D2C002309F457C090
:1030B00004E7402E0AE2502E40912D2C50E008E605
:1030C00011E00E94B33BA801569D502D479D500D25
:1030D000469D402D510D4A0D5B1D483601E05007BD
:1030E00014F0485651408401292D220F220B322F13
:1030F0000E945C3CC801D9018A01252F220F220BB6
:10310000322F0E945C3CA801B90105E31AEF2EE8BA
:103110003CE30E941C3D0E943242AC01BD010E9472
:103120001C3DC801D9018401292D220F220B322F09
:103130000E945C3CAC01BD010E94BB3C0E94693C0A
:10314000F201019311932F0101E0600E00E0701E67
:1031500000912D2C10E0601671060CF4ADCF0C948C
:10316000270F5A924A92BA93AA939A938A93502E0F
:103170000091BF2B1091C02B0536104008F4F9C008
:103180004090402C01E0A4D401E00093402C20E0CA
:1031900030E000E010E077DF00E00093162C0093B1
:1031A000172C0093182C0093192C0091B026109125
:1031B000B12600936A2C10936B2C85D10CE07FD73D
:1031C00080E098EEADE7B7E480936C2C80936D2C93
:1031D0002091B0263091B12600916C2C10916D2C6D
:1031E00052DF03E06CD70091BF2B1091C02B1A93D4
:1031F0000A932EE433E20AE818E20E94E54222969E
:103200002AE838E212E306E00E94930F0091BF2BF8
:103210001091C02B20E030E00E94673CAC01BD0162
:103220000E941E3EC8F40091BF2B1091C02B20E0DD
:1032300030E00E94673CC801D90100916C2C1091CC
:103240006D2C0093682C1093692CE091BF2BF091AA
:10325000C02B799708F467C0ECE6FCE2008111818D
:103260000B5F1F4F00831183083611400CF4B0CF61
:1032700080E098EEADE7B7E40AE010E0F8D004E6AD
:103280000093B0268093B1262091B0263091B126CC
:103290000091682C1091692CF6DE03E010D70091A4
:1032A000BF2B1091C02B1A930A932EE433E20AE845
:1032B00018E20E94E54222962AE838E212E306E08C
:1032C0000E94930F0091BF2B1091C02B20E030E0A3
:1032D0000E94673CAC01BD010E941E3EC0F40091FB
:1032E000BF2B1091C02B20E030E00E94673CC8014A
:1032F000D9010091B0261091B12600936A2C109349
:103300006B2CE091BF2BF091C02B749760F0E0EB39
:10331000F6E2008111810C5E1F4F00831183003D96
:1033200017400CF4B1CF20916A2C30916B2C285FA0
:103330003F4F0091682C1091692CA5DE00916A2CFA
:1033400010916B2C0093182C1093192C0091682C61
:103350001091692C0093162C1093172C552009F00E
:1033600009D04092402C0091402CB2D300E61AEED6
:10337000B1D617CE2091172C0EE010E0D6D92091AF
:10338000162C0FE010E0D1D92091192C00E110E0AB
:10339000CCD92091182C01E110E0C7C93091482CFC
:1033A000329F23E3021620E012061CF022E3022ED5
:1033B000112400922A0810922B08009326081093DB
:1033C000270808953091472C329FF3CFBA93AA93E0
:1033D0009A938A93D80184E090E0E091472CF0E042
:1033E0003197F89FF02DE99FF00DE89FF10D0092C5
:1033F0002A08F0932B08A0932608B093270808EE1C
:103400001DEF68D608EE1DEF65D600E315E762D61E
:103410000197813000E0900704F789919991A99173
:10342000B9910895BA93AA939A938A93D80188E0A0
:1034300090E0E091472CF0E03197F89FF02DE99F64
:10344000F00DE89FF10D00922A08F0932B08A0934D
:103450002608B093270808EE1DEF3CD608EE1DEFB6
:1034600039D60197813000E090071CF7D6CF209124
:10347000472C30E020932A0830932B0824E6219F24
:10348000302D209F310D009226083093270848E701
:1034900050E00091B62B1091B72B0E94B33B0395DF
:1034A0000ED600E000932A0800932B0808958A9313
:1034B000812F10E0DCDF00E315E70CD6082F10E0C9
:1034C000D6DF899108950E944C0E26E533E20AE882
:1034D00018E20E94E5422AE838E21AE003E00E947E
:1034E000340F00E310E0C3CF0E94C93A40E050E03F
:1034F00064E672E40E941C3D0C94693C7A926A92E4
:103500005A924A92BA93AA939A938A93C801D9017C
:103510002A013B010091252C10E020E030E00E94C0
:10352000673CA801B901820193010E94953DAC015D
:10353000BD010E94BB3CA201B3010E94C93A40E018
:1035400050E064E672E40E941C3D0E94693CC801A0
:1035500000913F2C073009F446968B3500E0900728
:103560001CF08AE590E006C0863A0FEF900714F44D
:1035700086EA9FEF8C0189919991A991B99149901F
:1035800059906990799008954A92BA93AA939A9320
:103590008A93A0E0B0E04090642CA093642CA093A8
:1035A0002202A093010202E08AD584EF91E004E1B7
:1035B00010E090D5E0E0F2E000810860008303A510
:1035C0000023E9F301E003A702891389A017B107DB
:1035D0000CF4D801019759F700E10183F09322021E
:1035E000A55DB04012F4A0E0B0E04092642C42E04F
:1035F00050E08D010E94B33B89919991A991B991B5
:1036000049900895E0E0F2E000810061008303A9A1
:103610000023E9F301E003AB4091442C50E000911A
:103620001402109115020C949B3B0091122C1091E6
:10363000132C3ADC0091122C1091132C74CC0091B5
:10364000122C1091132C30DC0091122C1091132CA1
:103650006ADC20914B2C06E4029F8001A9DC0091DA
:10366000B62B1091B72B00932609109327090895C4
:103670009A938A9301E010E00E945513902F02E084
:1036800010E00E94551310E00093B62B9093B72BD7
:1036900005E00E945513902F06E010E00E9455139C
:1036A0000093122C9093132C0DEF11E00E945513F0
:1036B00000933F2C073089F4E091122CF091132CE9
:1036C0007997E2E1FCE2008111811CF00951104080
:1036D00002C0015B1E4F0083118307E010E00E94CF
:1036E0005513902F08E010E00E94551310E000934E
:1036F000142C9093152C0EE00E945513902F0FE080
:1037000010E00E94551310E00093162C9093172C94
:1037100000E10E945513902F01E110E00E94551323
:1037200010E00093182C9093192C03E00E9455137D
:103730000093412C0CE110E00E9455130093422CA1
:1037400004E110E00E9455130093402C09EF11E0B2
:103750000E9455130093432C07EF11E00E9455136C
:1037600000934A2C0CE010E00E94551300934B2C60
:103770000CEF11E00E9455130093442C06EF11E06A
:103780000E9455130093462C0BEF11E00E94551335
:103790000093242C0DEF11E00E94551300933F2C51
:1037A0000DE010E00E9455130093492C0AE010E050
:1037B0000E945513802F0BE010E00E945513809358
:1037C000542C0093552C09E110E00E9455130093EE
:1037D0002A2C02E110E00E94551300932B2C08EFD5
:1037E00011E00E9455130093352C0BE110E00E946C
:1037F000551300933E2C09EE11E00E9455130093DF
:10380000272C08EE11E00E9455130093282C0091FC
:103810003F2C023019F400E00093422C0FEF11E02E
:103820000E94551300932C2C023028F020E00FEF5B
:1038300011E00E94951300913F2C053049F403E0FC
:103840000093492C04E000933E2C01E00093402CAF
:10385000E4E5FCE20C94620E9A938A9381E0009175
:10386000B82B00230AF463C04AE00E947D3B402F3E
:103870004A5F0091542C1091552C0E94953B017089
:1038800009F0A0C020912A2C30E00091B82B102F15
:10389000110F110B201731070CF494C000914A2C22
:1038A000013029F42091342C08E51BE18AC0023054
:1038B00081F40091B82B02332CF42091342C00EBCE
:1038C00016E37FC00B3474F32091342C0CEA1DE016
:1038D00078C00330C9F42091342C8BE090E0009143
:1038E000B82B102F110F110B4AE050E00E94B33B90
:1038F000801B910B04E115E0189F102D099F100DFE
:10390000089F002D110D5DC0043009F05BC02091AF
:10391000342C4EE650E00091B82B102F110F110BF4
:10392000401B510B02E8059F102D049FEACF009128
:10393000422C10E020911C2C30911D2C02171307F3
:103940000CF040C094E04CEE0091B82B0E947D3BFF
:10395000901B492F0091542C1091552C0E94953B9F
:10396000017081F50091342C06950093342C009160
:103970004A2C023008F082E000913F2C0230C9F45A
:1039800020911A2C30911B2C00E510E04091402C26
:1039900052E0459F001911092017310754F4209176
:1039A000342C08E51BE1189F102D089F002D110DE8
:1039B00008C00091B82B023F94F72091342C00EE00
:1039C0001BEAECDC8991999108954A92BA93AA93E3
:1039D0009A938A930CE00093462CE4E2F6E000818F
:1039E0000D7F008305E06BD30091272C10E00E942F
:1039F000AB1223E633E20AE818E20E94E54200E84F
:103A00000E94C010AAE1B4E088E59BE102E2402EEA
:103A100029E08C01D7DC00E315E75CD3A0936A09A9
:103A2000B0936B09885C90405E974A9489F7009147
:103A3000880603FFE7CF09E142D30091880603FF20
:103A4000E1CF0E944C0E21E733E20AE818E20E941F
:103A5000E5422AE838E21AE003E00E94340F00E56C
:103A600010E005DD0CE310E002DD08E210E0FFDC11
:103A7000E4E8F6E000810B7F008304E110E0F7DC6E
:103A80000091880603FDFCCFBDCF8A930E944C0EA7
:103A90000091392C0023D1F4B5DD04321040B4F488
:103AA00080E027E733E20AE818E20E94E542082FA7
:103AB00000580E94C01008E710E0D9DC08EB18E8B5
:103AC00009D302E0FCD28395853058F3899108959B
:103AD00010912002137E109320020A95000F000F10
:103AE00010912002102B1093200200E21EE4F2D26B
:103AF00001E00093312C0895BA93AA939A938A9384
:103B00008091B62B9091B72B0196AC01692F660F6F
:103B1000660B762F00E01CE62CED32E00E94FA3BAB
:103B200040912D2C50E060E070E00E94FA3BC8010B
:103B3000D90148EE53E060E070E00E94FA3B085083
:103B400000934C2C80935A2C90935B2C00912D2C3D
:103B500040E00B9F302D0A9F202D310D099F102D25
:103B6000210D341F089F002D110D241F341F42E723
:103B700050E060E070E00E94FA3B007E0093C52BAD
:103B80001093C62B0091642C002311F44FE301C065
:103B900041E250E00091C52B0E949B3B0093C72B54
:103BA0001093C82B0091C52B1091C62B0093C32BEB
:103BB0001093C42B47E150E00091B62B1091B72B26
:103BC0000E94B33B0093C92B1093CA2B26CC50DD27
:103BD0000091642C002341F400E100932D2CE4E2D9
:103BE000F6E00081016007C008E000932D2CE4E2BC
:103BF000F6E000810E7F00830091462C0093472C55
:103C00007BDF2091182C3091192C0091162C1091EB
:103C1000172C39DA14DD0091402C5ADF94C022E0D1
:103C20002093CA01F801049000E00093CA01002D1E
:103C30000895BA93AA939A938A93A0E090E088E0BB
:103C40008C01EDDFB02F8C010F5F1F4FE8DFB09FBD
:103C5000A00D83958D30A0F388E0082F10E0DFDF02
:103C6000900F83958431C8F3AA2309F4A3E0992324
:103C700011F09F3F09F4A7E0192F0A2FCECB9A939A
:103C80000BEE11E00E9455130F3F31F50CEE11E0E1
:103C90000E9455130F3F01F5CCDF912F202F0CEE22
:103CA00011E00E949513292F0BEE11E00E9495134D
:103CB00020E00DEE11E00E94951320E00EEE11E0E1
:103CC0000E94951300E00093CD2B0093CE2B20E0B3
:103CD00003EF11E00E94951399910895282F412F29
:103CE000802F849F802D800F895F480F802F849FB5
:103CF000802D840F800F8D5F082F142F822F089541
:103D0000392F482F212F802F829F802D810F800FE8
:103D1000875F982F2FEF201B822F8C01842F932FEA
:103D2000089500EB0093010202E20093020203E017
:103D3000009304020093200208E200932102E0E0D5
:103D4000F2E00C94EB0D00913F2C002341F401E0D4
:103D500010E80093542C1093552C02E023C001303E
:103D600011F40FE119C0023091F3033041F40FE078
:103D700010E80093542C1093552C01E013C004302C
:103D800041F40FE510E80093542C1093552C0AE0F1
:103D900009C0053051F40FE010E80093542C109343
:103DA000552C04E00093252C0895063041F40FEDC6
:103DB00018E90093542C1093552C00E1F3CF0730F1
:103DC00049F403E010E80093542C1093552C05E0BF
:103DD0000093252C0895053080F401E00093672AB4
:103DE00003E00093682A05E00093692A07E0009346
:103DF0006A2A00E000936B2A11C009F500E00093E5
:103E0000672A01E00093682A03E00093692A05E02D
:103E100000936A2A07E000936B2A00E000936C2A63
:103E200000936D2A00936E2A00936F2A0093702AE4
:103E30000093712A0093722A0093732A0895063022
:103E400099F400E00093672A0093682A01E0009348
:103E5000692A03E000936A2A05E000936B2A07E0D1
:103E600000936C2A00E0DCCF0730A9F400E0009357
:103E7000672A0093682A0093692A01E000936A2A5E
:103E800003E000936B2A05E000936C2A07E000939F
:103E90006D2A00E0C7CF0830B9F400E00093672A2C
:103EA0000093682A0093692A00936A2A01E000932C
:103EB0006B2A03E000936C2A05E000936D2A07E06B
:103EC00000936E2A00E0B0CF0930C9F400E00093FF
:103ED000672A0093682A0093692A00936A2A00934C
:103EE0006B2A01E000936C2A03E000936D2A05E041
:103EF00000936E2A07E000936F2A00E097CF0A3004
:103F0000D9F400E00093672A0093682A0093692A95
:103F100000936A2A00936B2A00936C2A01E00093B5
:103F20006D2A03E000936E2A05E000936F2A07E0F4
:103F30000093702A00E07CCF0B30E9F400E000939E
:103F4000672A0093682A0093692A00936A2A0093DB
:103F50006B2A00936C2A00936D2A01E000936E2A6D
:103F600003E000936F2A05E00093702A07E00093B6
:103F7000712A00E05FCF0C30F9F400E00093672A6B
:103F80000093682A0093692A00936A2A00936B2A97
:103F900000936C2A00936D2A00936E2A01E000932F
:103FA0006F2A03E00093702A05E00093712A07E06E
:103FB0000093722A00E040CF0D30F9F400E0009346
:103FC000672A0093682A0093692A00936A2A00935B
:103FD0006B2A00936C2A00936D2A00936E2A00933B
:103FE0006F2A01E00093702A03E00093712A05E034
:103FF0000093722A07E00093732A08950091432CDE
:10400000002311F00AE201C000E200930F2C089592
:104010008A934091402C4E5FEFEEFBE200811181CC
:10402000228133810E94CF3B0093222C4091402C6F
:104030004E5FE7EFFBE200811181228133810E9414
:10404000CF3B0093232C102F110F110B0E94C13A6C
:104050000731104094F50091222C102F110F110BF5
:104060000E94C13A0034104044F50091B82B00235F
:104070008AF00091232C102F110F110B0E94C13ACE
:10408000802F0091222C102F110F110B0E94C13A8A
:10409000182F11C00091222C01301CF001950093C3
:1040A000222C0091232C102F110F110B0E94C13ACA
:1040B000102F0091222C0E94030E899108958A935B
:1040C000802FA89503C008EE1DEF04D08A95D9F77C
:1040D000899108959C01C8010197F1F7C8010197E2
:1040E000F1F743E050E00E949B3BC8010197F1F7D4
:1040F000C9010895DA92CA92BA92AA929A928A92C1
:104100007A926A925A924A92BA93AA939A938A930B
:104110002397F89403E00E94470DE0E8F6E0008161
:1041200004600083009160060F6300936006E0E482
:10413000008101600083008102600083E0E2008171
:1041400001600083008102600083E0E4008104607C
:10415000008308E1048B058B068B078B038B08E239
:10416000AEDFE4E8F6E00081046000830E94AC0D5D
:104170000E944C0E00EF11E00E9455130F3F11F406
:1041800081E001C080E001EF11E00E9455130F3F74
:1041900011F401E001C000E0802351F020E000EFC5
:1041A00011E00E94951320E001EF11E00E949513A9
:1041B0000AEF11E00E9455130F3F11F401E001C016
:1041C00000E0E8E4F6E0108115FD08C0108116FD5E
:1041D00005C0108114FD02C011E001C010E0012BE8
:1041E00009F4F5C00E944C0E27E833E20AE818E211
:1041F0000E94E54200EC0E94C01003EF11E00E9413
:1042000055130A3050F024E003EF11E00E9495139B
:1042100020E002EF11E00E94951300E00093652C6E
:1042200000E00093642C02C0002351F421E001E07F
:1042300010E00E94951326E702E010E00E9495131B
:104240000091642C013051F421E001E010E00E9463
:1042500095132FE802E010E00E94951320E005E09E
:1042600010E00E94951324EB06E010E00E949513E5
:1042700020E007E010E00E94951320EB08E010E03A
:104280000E94951320E00EE010E00E94951320E0BC
:104290000FE010E00E94951320E000E110E00E9482
:1042A000951320E001E110E00E94951326E003E061
:1042B00010E00E94951321E00CE110E00E9495139C
:1042C00022E004E110E00E94951321E00BEF11E0E1
:1042D0000E94951325E009EF11E00E9495132AE052
:1042E0000CE010E00E94951321E00DE010E00E9428
:1042F000951321E007EF11E00E94951321E00AE0F9
:1043000010E00E94951320E80BE010E00E94951346
:104310002FE20CEF11E00E94951321E008EF11E06D
:104320000E94951325E006EF11E00E94951320E00E
:104330000DEF11E00E94951327E509E110E00E94BE
:10434000951327E00BE110E00E94951320E005EFA4
:1043500011E00E9495130AE010E061DCA02FA29505
:10436000A07FA03509F4A0E92A2F0AEE11E00E94EF
:10437000951324E609EE11E00E94951320E008EE63
:1043800011E00E94951320E002E110E00E949513D5
:1043900021E00FEF11E00E9495130091642C03952A
:1043A0000093642C033008F43FCF0091652C0395F3
:1043B0000093652C043008F433CF20E00AEF11E0BD
:1043C0000E94951320E004EF11E00E9495130AEF7C
:1043D00011E00E9455130093652C04EF11E00E9438
:1043E00055130093642CF3DB0091282C0023E4E2A6
:1043F000F6E0008139F402600083E4E400810160AA
:1044000000830EC00D7F0083E4E400810E7F0083F3
:1044100000E61AEE5FDE0091272C10E00E94AB123E
:104420000EE14DDE03E20093010804E00093000872
:1044300000E000932A0800932B0803E2009341094F
:1044400006E00093400908EE13E00093660910931C
:1044500067092091432C04E6029F00926A0910929A
:104460006B090091432C002329F400E000936609B6
:104470000093670901E0009300090091B62B1091A9
:10448000B72B009326091093270903E00093060930
:104490000091A20007600093A20007E0009340088B
:1044A00004ED11E000936608109367081093460826
:1044B0000E94740D00919300043019F400E1009300
:1044C00022039CDD2EDC00E210E0A9DB00930C024D
:1044D00001E210E0A4DB00930D0202E0009322024F
:1044E0000E946D0D0E94660DAAD80091480607FF34
:1044F0006CDA0E944C0E27E933E20AE818E20E94C7
:10450000E5422DE933E215E001E00E94340F05E0B9
:10451000D6DD00ED17E00E94E61900ED17E00E94DD
:10452000E6192FE933E215E102E00E94340F00EAB8
:104530001FE00E94E61921EA33E215E201E00E9441
:10454000340F00E41FE10E94E61923EA33E215E389
:1045500002E00E94340F00E513ECBCDD08E813E133
:104560000E94E61900E000932A0800932B080EE150
:10457000A6DD25EA33E212E401E00E94340F08E8E8
:1045800013E10E94121A00E000932A0800932B08FE
:1045900000918A280B3409F0A8CF00918B280035B0
:1045A00009F0A3CF00918C280F3409F09ECFA0E032
:1045B0001CE10A2F0E94D50FA395A038C8F30091E3
:1045C0008D28043509F091CF00913F2C12E0019F16
:1045D00000912C2C10E0000E111E000C111CF0019B
:1045E000E750F74E059114911A930A932BEA33E2A0
:1045F0000AE818E20E94E54222962AE838E219E128
:1046000005E00E94340F0091282C013091F40091B4
:10461000272C10E01A930A932EEA33E20AE818E2F4
:104620000E94E54222962AE838E21FE007E00E9455
:10463000340F07E344DD08ED04BF0BE20093800074
:104640000091820000FDFCCF0E94E412E3EAF6E252
:10465000408151816281738104171507260737074E
:1046600039F10E944C0E2BEB33E20AE818E20E946B
:10467000E54200EC0E94C010E8E4F6E0008105FD90
:1046800016C0008106FD13C00E94E4123A932A93DB
:104690001A930A932AEC33E20AE818E20E94E542F0
:1046A00024962AE838E218E206E00E94930FFFCF32
:1046B0000BEE11E00E945513902F0CEE11E00E94BA
:1046C00055130093CB2B9093CC2B0DEE11E00E9451
:1046D0005513902F0EEE11E00E9455130093CD2B31
:1046E0009093CE2B0091CB2B1091CC2B09DB2091FA
:1046F000CD2B3091CE2B02171307A1F420E50AEE43
:1047000011E00E9495132FEF0BEE11E00E9495131C
:104710002FEF0CEE11E00E94951308ED04BF01E0AD
:10472000009379000BEE11E00E945513902F0CEED0
:1047300011E00E9455130093CB2B9093CC2B0DEEE0
:1047400011E00E945513902F0EEE11E00E945513B8
:104750000093CD2B9093CE2B0091CB2B1091CC2B93
:10476000BDDA2091CD2B3091CE2B0217130779F4AF
:1047700060DA2091CB2B3091CC2B0217130739F440
:1047800002E000934E2C04E000934F2C59C001EF3F
:1047900011E00E9455130230F8F501E000934E2C11
:1047A0000E944C0E2EEC33E20AE818E20E94E54229
:1047B00000E80E94C0102DED33E20AE818E20E94E2
:1047C000E5422AE838E215E007E00E94930F00EF87
:1047D00011E00E945513802F01EF11E00E94551344
:1047E000202F0CE310E0081B10401A930A9301E0FD
:1047F00010E0021B10401A930A9321EF33E20AE8FB
:1048000018E20E94E542249600EC0E94C01004E6E3
:1048100056DC04E654DC14C004E000934F2C0CE09A
:1048200000932F2C0FEF0093392C02E000933A2CC9
:104830000DE40093372C00E00093A40800934E2C65
:10484000789408EE1DEF46DC20D90091402C40D929
:10485000E8E4F6E0008105FD23C0008104FD20C0EE
:104860000FEF0093392C0EE00093372C01E00093FA
:104870003A2C0E944C0E23E034E20AE818E20E942F
:10488000E5422AE838E211E001E00E94340F10E529
:1048900000E30E94571A0091480604FDF6C0FBCFC2
:1048A000008104FD1AC00FEF0093392C02E0009341
:1048B0003A2C0E944C0E10E500E30E94571A24E1A6
:1048C00034E20AE818E20E94E5422AE838E21AE0F7
:1048D00001E00E94340F0DE4D6C0008106FDB1C096
:1048E00002E316C000914B2C039500934B2C05312D
:1048F00038F004E100934B2C00E510E00E94371AD9
:1049000020914B2C06E4029F80010E94D81706E4F8
:1049100010E00E94371A0E944C0EA091402C01E03A
:104920000093402CD5D80AE0CADB0E94C41A380193
:104930000091BF2B1091C02B053E2CE01C4028F0AD
:1049400004EE0093BF2B2093C02BA89500915A2C06
:1049500010915B2C1A930A9320E234E20AE818E2E1
:104960000E94E542229600E80E94C0107A926A9264
:104970002CE234E20AE818E20E94E542229600ECBA
:104980000E94C0100091BF2B1091C02B1A930A9364
:104990002CE334E20AE818E20E94E54222962AE873
:1049A00038E213E205E00E94E90E22E434E20AE86C
:1049B00018E20E94E5422AE838E21CE607E00E947D
:1049C000340F0AE07CDBE8E4F6E0008104FF8ACFE4
:1049D000008105FD13C000914B2C0A9500934B2CD0
:1049E0000F3F19F400E000934B2C20914B2C06E470
:1049F000029F80010E94D8170CE38ACF008106FD38
:104A000016C00091642C002311F401E001C000E005
:104A10000093642CDCD800E510E00E94371A06E40D
:104A200010E00E94371A01E00093312C74CF00810E
:104A300007FD7DC000E410E00E94371AC8D8A0939B
:104A4000402C0091C92B3BDB0E94C41A053010405A
:104A5000CCF40E944C0E26E434E20AE818E20E94EC
:104A6000E54200EC0E94C01000ED10E00E94371AF1
:104A700000EB10E00E94371A00ED10E00E94371A98
:104A800008E01DDB00E00093372C0091880603FD51
:104A9000FCCF02EF11E00E945513073381F00E9412
:104AA000C41A8091BF2B809F802D002D023411F0FD
:104AB000863629F42FEF0AEF11E00E94951301E0EA
:104AC0000093312C0AE000933D2C00933C2C00E035
:104AD0000093B92B01E010E00093562C1093572C53
:104AE00000933B2C00E30E94371A02E0E8DA00E36F
:104AF00010E00E94371A0CE000932F2C01E0009385
:104B0000382C0093312CCC2400E6D02E00914E2C72
:104B10000B5F0093292C0E944C0E01E00093302C77
:104B20000091372C58D90E94300E0C941B32E8E8C3
:104B3000008103FFFDCE09E1C2DA0091880603FF80
:104B4000F7CE0E944C0E21E733E20AE818E20E94F9
:104B5000E5422AE838E21AE003E00E94340F00E55B
:104B600010E00E94371A0CE310E00E94371A08E2A6
:104B700010E00E94371AE4E8F6E000810B7F008322
:104B800004E110E00E94371A0091880603FDFCCF73
:104B9000CFCE202F239500EF11E00E94D813009173
:104BA0004E2C023088F401EF11E00E9455130230C0
:104BB00058F00FEF0093392C02E000933A2C0DE4EB
:104BC0000093372C0E944C0E00913A2C002309F0E0
:104BD000DBC30AE01091412C011B000F000F000FF6
:104BE00010912B2C010F0093502C0091452C01307B
:104BF00009F000C200913B2C013009F0FBC100E03C
:104C00000093452CE7EDFBE2008111812281338185
:104C1000EFEEFBE20083118322833383EBEDFBE2B3
:104C20000081118122813381E7EFFBE20083118350
:104C3000228333830E945C3C48015901EFEEFBE282
:104C400000811181228133810E945C3C5091642C4F
:104C500044E0549FF001E855F94D00801180228016
:104C60003380A801B901800191010E941C3DA80177
:104C7000B901840195010E94FF3C0E94693C0093A8
:104C80001A2C10931B2C00913F2C043059F4EFEE9A
:104C9000FBE200811181228133813595279517959B
:104CA000079502C00AE510E000931E2C10931F2CFC
:104CB00000911A2C10911B2C0E5F1F4F212F220FD9
:104CC000220B322F0E945C3C0E94B23E0E94693C43
:104CD00010E000931C2C10931D2C0091502C102FD1
:104CE000110F110B20911A2C30911B2C0217130756
:104CF0000CF052C1102F110F110B20911E2C30916E
:104D00001F2C021713070CF047C100E000933C2C46
:104D100000913D2C039500933D2C053118F001E0E6
:104D20000093312CE3EFFBE200811181228133817A
:104D3000EFEEFBE24081518162817381401B510B98
:104D4000620B730B4083518362837383EBEFFBE24F
:104D50000081118122813381E7EFFBE240815181A3
:104D600062817381401B510B620B730B4083518333
:104D700062837383EFEEFBE2408151816281738134
:104D80008A019B012224349F302D259F300D300D48
:104D9000079F300D249F202D310D159F200D311DB3
:104DA000069F200D311D149F102D210D321D100D59
:104DB000211D321D049F002D110D221D321DE7EF14
:104DC000FBE280809180A280B380A401B501789D30
:104DD000702D699D700D700D4B9D700D689D602D3F
:104DE000710D599D600D711D4A9D600D711D589D7D
:104DF000502D610D721D500D611D721D489D510D8C
:104E0000621D721D000D151F261F371F0E945C3C7E
:104E10000E9400430E94693CC8019595879595952D
:104E2000879599236AF426E000E114EA0E94E219CA
:104E300000ED17E04FD906E00093342C0E942C1CA3
:104E40000091472C0093482C8C01292F220F220B14
:104E5000322F0E945C3C0E94B23E0E94693C00934B
:104E6000BE2BE7EFFBE200811181228133810E949A
:104E70005C3CA801622FB32EEFEEFBE200811181B2
:104E8000228133810E945C3C7B2D0E947E1A00931C
:104E9000B82B0093BD2B09811A8120911A2C3091D7
:104EA0001B2C0217130754F40091B82B0093BA2B54
:104EB0008093562C9093572C29833A830091B82BDA
:104EC0001091BC2B011714F40093BB2B0091BB2B4A
:104ED0000093BC2B0091BA2B0093B82B0091352C7A
:104EE000002311F408E047C0013019F400911C2C94
:104EF00042C00230E1F46090472C85E090E042E04F
:104F000050E000911C2C10911D2C0E94B33B801B83
:104F1000910BAC01062D10E00E94B33B0093482C8E
:104F2000002319F401E00093482C48E01DC0033031
:104F300021F56090472C85E090E042E050E0009140
:104F40001C2C10911D2C0E94B33B801B910BAC01BB
:104F5000062D10E00E94B33B0093482C002319F467
:104F600001E00093482C40E150E000911A2C109190
:104F70001B2C0E94B33B0093342C00912B2C12E08D
:104F8000019F00911A2C10911B2C001611060CF099
:104F9000D5C10E942C1CD2C100E000932A080093C6
:104FA0002B08EFEEFBE20081118122813381E3EFD8
:104FB000FBE20083118322833383E7EFFBE200816E
:104FC000118122813381EBEFFBE200831183228385
:104FD000338300E00093BE2B10E009830A830AE5C7
:104FE0000093BB2B00913C2C039500933C2C109319
:104FF0003D2CA4C100913B2C002309F09FC1E7ED9B
:10500000FBE20081118122813381EFEEFBE200831C
:10501000118322833383EBEDFBE200811181228136
:105020003381E7EFFBE200831183228333830E9405
:105030005C3C48015901EFEEFBE2008111812281C5
:1050400033810E945C3C5091642C44E0549FF001F9
:10505000E855F94D0080118022803380A801B90104
:10506000800191010E941C3DA801B90184019501B4
:105070000E94FF3C0E94693C00931A2C10931B2C49
:1050800000913F2C043059F4EFEEFBE200811181D6
:1050900022813381359527951795079502C00AE53A
:1050A00010E000931E2C10931F2C00911A2C1091CD
:1050B0001B2C212F220F220B322F0E945C3C0E94BE
:1050C000B23E0E94693C00931C2C10931D2C8091D1
:1050D000502C982F990F990B029600911A2C109131
:1050E0001B2C801791070CF0FEC08091502C982F3C
:1050F000990F990B029600911E2C10911F2C80176E
:1051000091070CF0F0C00091372C002309F0EBC0A0
:1051100000E000933C2C00913D2C039500933D2C26
:10512000E3EFFBE20081118122813381EFEEFBE2AC
:105130004081518162817381401B510B620B730B63
:105140004083518362837383EBEFFBE20081118123
:1051500022813381E7EFFBE24081518162817381DB
:10516000401B510B620B730B40835183628373832B
:10517000EFEEFBE240815181628173818A019B01E4
:105180002224349F302D259F300D300D079F300D88
:10519000249F202D310D159F200D311D069F200DC0
:1051A000311D149F102D210D321D100D211D321D9A
:1051B000049F002D110D221D321DE7EFFBE28080C0
:1051C0009180A280B380A401B501789D702D699D66
:1051D000700D700D4B9D700D689D602D710D599D6A
:1051E000600D711D4A9D600D711D589D502D610D02
:1051F000721D500D611D721D489D510D621D721D65
:10520000000D151F261F371F0E945C3C0E940043A3
:105210000E94693CC80195958795959587959595C8
:1052200087959595879599234AF424E004E016EA3A
:105230000E94E21900EA1FE00E946A200091472CB8
:105240000093482C00913D2C063098F100912B2CB6
:1052500012E0019F00911A2C10911B2C00161106D0
:1052600044F520911C2C00E81EE340911A2C50912B
:105270001B2C5595479555954795041B150B0E947A
:10528000E219E7EFFBE200811181228133810E9464
:105290005C3CA801622FB32EEFEEFBE2008111818E
:1052A000228133810E945C3C7B2D0E947E1A0093F8
:1052B000B82B09811A8120911A2C30911B2C0217CE
:1052C000130754F40091B82B0093BA2B8093562CFB
:1052D0009093572C29833A830091BA2B0093BC2BCF
:1052E0000093B82B2BC000E000932A0800932B08F2
:1052F000EFEEFBE20081118122813381E3EFFBE2DB
:105300000083118322833383E7EFFBE20081118165
:1053100022813381EBEFFBE200831183228333830D
:1053200000E009830A830093562C0093572C0093C6
:105330003D2C00913C2C039500933C2C00913C2C7F
:10534000003F21F000913D2C003F99F400E010E077
:105350000093562C0093572C0093B92B0093B82B35
:105360000093BD2B0093BE2B01E00093312C1093D2
:10537000522C00913C2C023C19F40E94300E04C0C7
:10538000083C11F40E9476100091392C002309F09A
:105390005BC20C2DC092662C07700093672C0091A5
:1053A000662C003319F40E94021B08830091662CBE
:1053B000093559F40091242C023039F0043029F0D9
:1053C0000E94761000E00093BD2B0091672C013005
:1053D00009F0AEC08091B82B982F990F990B0091CE
:1053E000562C1091572C0D5F1F4F212F220F220B8F
:1053F000322F0E945C3C0E94B23E40E050E060E8E8
:105400007FEB0E94BB3C0E94693C28010091562C16
:105410001091572C0093582C1093592C00911A2C52
:1054200010911B2C0D3310400CF4C2C0082F809338
:10543000B92BA201192F0E94B33B42E050E00E9419
:10544000B33B102F110F110B38010091BA2B102F05
:10545000110F110B2091BC2B322F330F330B021B7A
:10546000130B0D5F1F4F212F220F220B322F0E9493
:105470005C3C0E94B23E0E94693CA80183010E94EC
:10548000B33B0093522C863500E0900724F4009142
:10549000BC2B00233AF442E00091522C0E947D3B49
:1054A0000093522CE0914C2CF0E0F3968E179F075E
:1054B0007CF000914C2C10E0005C1F4F081719077E
:1054C0003CF042E00091522C0E947D3B0093522C14
:1054D000552012F400E007C00091522C0023D2F3B3
:1054E0000B301CF00AE00093522C0091522C102F2C
:1054F000110F110B2091A726322F330F330B021BF4
:10550000130B42E050E00E94B33B1091A726010F1D
:105510000093522C0093A726840D951D892B19F416
:1055200000E00093522C0091522C0093512C40C06B
:105530000230F1F50091202C0075093210F00AE3D9
:1055400001C000E20093102C00EF11E00E945513FF
:10555000802F01EF11E00E94551390E09A938A93F7
:105560002091102C9A932A939A930A9324E534E27B
:105570000AE818E20E94E54226962AE838E21AE391
:1055800003E00E94930F0091182C1091192C012B0D
:1055900019F02FE534E202C027E634E20AE818E207
:1055A0000E94E5422AE838E21EE503E00E94930FDC
:1055B0000091292C073091F022E433E20AE818E246
:1055C0000E94E5422AE838E215E507E00E94930FC1
:1055D0002AE838E214E107E00E94930F0091672C5B
:1055E000033009F048C04AE008810E946F3B50E058
:1055F0005A930A924AE00A810E946F3B5A930A9397
:1056000000910F2C5A930A930091492C5A930A93B4
:105610000091412C5A930A930091402C5A930A937B
:105620002EE634E20AE818E20E94E5422C962AE8C7
:1056300038E21AE301E00E94930F00915A2C109176
:105640005B2C1A930A9300913E2C10E01A930A9354
:105650008091652C90E001969A938A9321E834E238
:105660000AE818E20E94E54226962AE838E21AE3A0
:1056700002E00E94930F0091672C043009F500911D
:10568000242C0430E9F00091B92B102F110F110BCD
:105690000E94C13A1A930A932EE834E20AE818E20B
:1056A0000E94E54222960091B92B00232AE838E2B5
:1056B00012E001E01AF00E94680E02C00E94A80EDB
:1056C00000913B2C013009F079C00091242C01306D
:1056D00041F50091672C063009F097C00091582CD5
:1056E0001091592C159507951595079515950795C2
:1056F0000E94C13A0093582C1093592CE091582CD9
:10570000F091592C789734F007E110E00093582C71
:105710001093592C1091582C0091BD2B0E942210EF
:1057200069C0023019F40E9408206BC0033089F56B
:10573000E7EFFBE200811181228133810E945C3C12
:10574000A801622FB32EEFEEFBE2008111812281CE
:1057500033810E945C3C7B2D0E947E1A980140910F
:10576000402C439500911A2C10911B2C0E94953BC4
:10577000802F07E0039F102D029F002D110D4AE09E
:1057800050E00E94B33B182F0E94E60F10E408E09F
:1057900033C00091BD2B102F110F110B1A930A93D8
:1057A00023E934E20AE818E20E94E54222962AE858
:1057B00038E21AE002E00E94340F23C00091672C07
:1057C000053011F40E947610E0911C2CF0911D2CF4
:1057D000319724F000911C2C0E948A1029E934E2B0
:1057E0000AE818E20E94E5422AE838E212E006E000
:1057F0000E94340F10E40A2F0E94EF0D0AEA0E9463
:10580000A40D0091242C043059F0A6E010E40A2FD6
:105810000E94EF0D0AEA0E94A40DA395A830B0F3F0
:105820000091672C073009F0FEC40E94B3102DE9E7
:1058300034E213E504E00E94930F0091522C000F14
:10584000000F0E94A310EFC400913A2C002309F02E
:1058500070C200912C2C12E0019FF001E753F74E2B
:10586000059114911A930A932BEA33E20AE818E29D
:105870000E94E54222962AE838E21AE00091672A5F
:105880000E94340F0091462C10E01A930A932FE9DE
:1058900034E20AE818E20E94E54222962AE838E259
:1058A0001FE50091672A0E94340F00912C2C12E012
:1058B000019FF001E353F74E059114911A930A9357
:1058C0002BEA33E20AE818E20E94E54222962AE82F
:1058D00038E21AE00091682A0E94340F0091352CBA
:1058E00010E01A930A932FE934E20AE818E20E94C2
:1058F000E54222962AE838E21FE50091682A0E94D4
:10590000340F00912C2C12E0019FF001EF52F74E62
:10591000059114911A930A932BEA33E20AE818E2EC
:105920000E94E54222962AE838E21AE00091692AAC
:105930000E94340FE0914A2C10E0F0E0E75EF64E52
:1059400004911A930A932FE934E20AE818E20E94BC
:10595000E54222962AE838E21FE50091692A0E9472
:10596000340F00912C2C12E0019FF001EB52F74E06
:10597000059114911A930A932BEA33E20AE818E28C
:105980000E94E54222962AE838E21AE000916A2A4B
:105990000E94340F0091262C10E01A930A93009174
:1059A0004B2C1A930A9325EA34E20AE818E20E9483
:1059B000E54224962AE838E210E300916A2A0E9420
:1059C000340F00912C2C12E0019FF001E752F74EAA
:1059D000059114911A930A932BEA33E20AE818E22C
:1059E0000E94E54222962AE838E21AE000916B2AEA
:1059F0000E94340F0091402C10E01A930A932FE973
:105A000034E20AE818E20E94E54222962AE838E2E7
:105A10001FE500916B2A0E94340F00912C2C12E09C
:105A2000019FF001E352F74E059114911A930A93E6
:105A30002BEA33E20AE818E20E94E54222962AE8BD
:105A400038E21AE000916C2A0E94340F00913E2C3B
:105A500010E01A930A9322EB34E20AE818E20E945B
:105A6000E54222962AE838E21FE500916C2A0E945E
:105A7000340F00912C2C12E0019FF001EF51F74EF2
:105A8000059114911A930A932BEA33E20AE818E27B
:105A90000E94E54222962AE838E21AE000916D2A37
:105AA0000E94340F00913F2C12E0019F00912C2C9A
:105AB00010E0000E111E000C111CF001E750F74E13
:105AC000059114911A930A932BEA33E20AE818E23B
:105AD0000E94E54222962AE838E212E300916D2AFC
:105AE0000E94340F00912C2C12E0019FF001EB5129
:105AF000F74E059114911A930A932BEA33E20AE8C0
:105B000018E20E94E54222962AE838E21AE0009163
:105B10006E2A0E94340F0AE010E02091422C021BF2
:105B200010401A930A9322EB34E20AE818E20E942A
:105B3000E54222962AE838E21FE500916E2A0E948B
:105B4000340F00912C2C12E0019FF001E751F74E29
:105B5000059114911A930A932BEA33E20AE818E2AA
:105B60000E94E54222962AE838E21AE000916F2A64
:105B70000E94340F0091432C10E01A930A932FE9EE
:105B800034E20AE818E20E94E54222962AE838E266
:105B90001FE500916F2A0E94340F00912C2C12E017
:105BA000019FF001E351F74E059114911A930A9366
:105BB0002BEA33E20AE818E20E94E54222962AE83C
:105BC00038E21AE00091702A0E94340F0091242CD0
:105BD000102F110F110B1A930A932FE934E20AE8E0
:105BE00018E20E94E54222962AE838E21FE5009179
:105BF000702A0E94340F00912C2C12E0019FF001BA
:105C0000EF50F74E059114911A930A932BEA33E261
:105C10000AE818E20E94E54222962AE838E21AE0F1
:105C20000091712A0E94340F00912A2C10E01A93DF
:105C30000A932FE934E20AE818E20E94E54222962C
:105C40002AE838E21FE50091712A0E94340F009182
:105C50002C2C12E0019FF001EB50F74E05911491AE
:105C60001A930A932BEA33E20AE818E20E94E5420B
:105C700022962AE838E21AE00091722A0E94340F34
:105C800000912B2C10E01A930A9322EB34E20AE8DD
:105C900018E20E94E54222962AE838E21FE50091C8
:105CA000722A0E94340F0091272C10E01A930A9355
:105CB00029EB34E20AE818E20E94E54222962AE83B
:105CC00038E21AE00091732A0E94340F0091282CC8
:105CD000002319F429EC34E202C02FEC34E20AE884
:105CE00018E20E94E5422AE838E21EE10091732A98
:105CF0000E94340FA1E025ED34E211E00A2F0E944A
:105D0000340FAE5FA830B8F30091372C000F0A951E
:105D10000093302C0091372C053018F007E00093E9
:105D2000302C27ED34E211E00091302C0E94340F2A
:105D30007AC2013009F087C10091372C0D500093D1
:105D4000302C0C2D0F71013029F40E94C41A0093DD
:105D5000262C11C00C2D0F71003169F44090BF2B1F
:105D60005090C02B0DE840160AE0500624F008EBD6
:105D7000402E0BE0502E00912C2C12E0019FF001E0
:105D8000E355F74E059114911A930A932BEA33E2E7
:105D90000AE818E20E94E54222962AE838E21AE070
:105DA00001E00E94930F8091652C90E001969A93F8
:105DB0008A9329ED34E20AE818E20E94E54222962D
:105DC0002AE838E21BE401E00E94930F0E94021BC4
:105DD000C80100912C2C12E0019FF001EF54F74E06
:105DE000059114911A930A932BEA33E20AE818E218
:105DF0000E94E54222962AE838E21AE002E00E9478
:105E0000930F4AE050E08C010E94B33B5A934A93AF
:105E10004AE050E08C010E94B33B1A930A932EEDA6
:105E200034E20AE818E20E94E54224962AE838E2C1
:105E30001BE402E00E94930F00912C2C12E0019FC2
:105E4000F001EB54F74E059114911A930A932BEA43
:105E500033E20AE818E20E94E54222962AE838E294
:105E60001AE003E00E94930F8091642C90E0019669
:105E70009A938A932FE934E20AE818E20E94E542F5
:105E800022962AE838E21BE403E00E94930F009177
:105E90002C2C12E0019FF001E754F74E059114916C
:105EA0001A930A932BEA33E20AE818E20E94E542C9
:105EB00022962AE838E21AE004E00E94930F00914B
:105EC0005A2C10915B2C1A930A930091262C10E007
:105ED0001A930A9328EE34E20AE818E20E94E54297
:105EE00024962AE838E21DE204E00E94930F009114
:105EF0002C2C12E0019FF001E354F74E0591149110
:105F00001A930A932BEA33E20AE818E20E94E54268
:105F100022962AE838E21AE005E00E94930F0091E9
:105F2000122C1091132C1A930A9324EF34E20AE8EE
:105F300018E20E94E54222962AE838E21BE405E0D6
:105F40000E94930F0091182C1091192C012B11F421
:105F5000A0E001C0A1E000912C2C12E0019FF00113
:105F6000EF53F74E059114911A930A932BEA33E2FB
:105F70000AE818E20E94E54222962AE838E21AE08E
:105F800006E00E94930F5A924A9202E0A09FF0010D
:105F9000E25EF64E059114911A930A932EEF34E2C5
:105FA0000AE818E20E94E54224962AE838E213E360
:105FB00006E00E94930F00912C2C12E0019FF0014B
:105FC000EB53F74E059114911A930A932BEA33E29F
:105FD0000AE818E20E94E54222962AE838E21AE02E
:105FE00007E00E94930F0091292C073019F42CE050
:105FF00035E202C027E135E20AE818E20E94E542F4
:106000002AE838E21AE008E00E94930FA1E025EDAB
:1060100034E211E00A2F0E94930FA395A930B8F340
:106020000091372C013149F0023139F0033129F068
:10603000053119F027ED34E202C028E235E211E023
:106040000091302CEAC0023009F0EDC000914E2CD6
:10605000023009F047C00E944C0E2AE235E20AE8FD
:1060600018E20E94E5422AE838E215E002E00E94C8
:10607000340F29E335E20AE818E20E94E5422AE8F3
:1060800038E21EE105E00E94930F02EF11E00E944A
:106090005513802F03EF11E00E94551390E09A935F
:1060A0008A939A930A930091CD2B1091CE2B1A9339
:1060B0000A9325E435E20AE818E20E94E5422696B2
:1060C0002AE838E21EE107E00E94930F07E30E94EE
:1060D0005F200E944C0E01E000933A2C05E10093F2
:1060E000372CA1C00E943F1E0BEE11E00E945513F9
:1060F000902F0CEE11E00E9455130093CB2B909340
:10610000CC2B00EF11E00E945513802F01EF11E01E
:106110000E94551390E09A938A939A930A9324E5E8
:1061200035E20AE818E20E94E54224962AE838E2BD
:1061300011E001E00E94340F0AEE11E00E945513B5
:106140009A930A930091CB2B1091CC2B1A930A931C
:1061500024E635E20AE818E20E94E54224962AE89D
:1061600038E219E501E00E94340F03EF11E00E94CC
:1061700055132091CD2B3091CE2B3A932A939A939D
:106180000A9329E635E20AE818E20E94E5422496DD
:1061900000EC0E94C0100C2D07700630A0F025ED19
:1061A00034E20AE818E20E94E5422AE838E2109157
:1061B0002F2C110F110F110F165003E00E94340FF6
:1061C00002E00E945F20A0E018E20A2F0E94D50F93
:1061D000A395AF37C8F32BE735E20AE818E20E942F
:1061E000E5422AE838E214E305E00E94930F22E832
:1061F00035E20AE818E20E94E5422AE838E215E0B2
:1062000007E00E94930F28E935E20AE818E20E94AD
:10621000E5422AE838E215E008E00E94930F08EE14
:106220001DEF0E946A2000E00093112CE8E4F6E0E4
:10623000008107FD28C100E000932A0800932B0885
:106240000091402C0E94681D0091372C0E94EB1E8B
:106250000091362C013089F40EE110E00E94371ACB
:106260000091480607FFFCCF08EC00933D2C0093FB
:106270003C2C00E00093362C94C00091480607FDAA
:106280003CC008EE1DEF0E946A200091112C03957E
:106290000093112C8091C92B9091CA2B01968017E5
:1062A000904058F70091392C00950093392C0E94AA
:1062B0004C0E0E94C41A0093262C01E00093362C49
:1062C00000E00093532C0091392C002339F400E0B6
:1062D0000093372C02E00E945F2004C00091382C0C
:1062E0000093372C00E000933A2C0AE510E00E945E
:1062F000371A01E00093312C4DC00091392C002356
:1063000021F501E00093312C0E944C0E00E010E0DA
:1063100000932A0800932B0800913B2C013031F4A4
:1063200010933B2C05E00E945F2003C001E0009326
:106330003B2C02E00E945F2001E00093312C0AEE2A
:1063400000933D2C00933C2C25C000913A2C013049
:1063500059F40091372C03950093372C0631A0F0A7
:1063600005E10093372C16C0023099F30091372CC9
:1063700003950093372C0E3018F001E00093372C72
:106380000091372C0E94EB1E0091372C0E3010F438
:106390000093382C08E210E00E94371A00E00093C6
:1063A000332CA8950091880603FF32C00FE00E94AD
:1063B0005F200091880603FF2BC00E944C0E22E94B
:1063C00036E20AE818E20E94E5422AE838E216E2DC
:1063D00003E00E94340F00E510E00E94371A0CE33E
:1063E00010E00E94371A08E210E00E94371AE4E831
:1063F000F6E000810B7F00830FE00E945F20E4E85D
:10640000F6E000810B7F0083E8E8008103FDFDCF0B
:1064100001E0C00E00E0D01E00E7D01664F0CC24EE
:10642000DD240091BF2B1091C02B083E134018F4BF
:1064300001E00093312C00914D2C013011F00C94AF
:10644000CF2500E000934D2C00EA0E948A0D0E94A7
:106450004C0E00EF11E00E945513A02F0B3310F4E7
:106460000C94C92501EF11E00E945513202F2395AC
:1064700001EF11E00E94951320E000EF11E00E946F
:1064800095130C94CF25008106FDF2C410E0109303
:106490002A0810932B0804E0009300080091372C81
:1064A0000023F1F00150D8F00C5008F42EC209F48A
:1064B0004DC20150A0F0035008F427C209F4D1C224
:1064C0000A9509F415C30A9509F4F2C30A9509F46B
:1064D0001CC20A9509F419C2085309F408C409CF6B
:1064E00000E315E70E946A200E944C0E0091292CBF
:1064F0000730A9F02BEA35E20AE818E20E94E542EB
:106500002AE838E21EE102E00E94340F00E910E0C0
:106510000E94371A00E910E00E94371AEDC100917D
:10652000480606FD10C000E513EC0E946A200091A9
:10653000112C03950093112C2091C92B3091CA2B5B
:106540002017304060F70091112C03950093112C17
:106550002091C92B3091CA2B2017304008F033C14D
:1065600000913F2C0730B0F024EB35E20AE818E246
:106570000E94E5422AE838E214E102E00E94340F6A
:1065800000EA10E00E94371A05E00E945F200E9496
:106590004C0E04CFE3EEFBE20081118122813381B6
:1065A0000E945C3CA801622FB32FEFEDFBE200815B
:1065B0001181228133810E945C3C7B2FCBD70093D9
:1065C000B82BEFEDFBE240815181628173818A013A
:1065D0009B012224349F302D259F300D300D079FC5
:1065E000300D249F202D310D159F200D311D069F4C
:1065F000200D311D149F102D210D321D100D211D58
:10660000321D049F002D110D221D321DE3EEFBE211
:1066100080819181A281B381AC01BD01789F702DF1
:10662000699F700D700D4B9F700D689F602D710DEF
:10663000599F600D711D4A9F600D711D589F502D0F
:10664000610D721D500D611D721D489F510D621D1F
:10665000721D000D151F261F371F0E945C3C0E94F3
:106660000043C801D901E3EEFBE2008111812281E0
:1066700033810E945C3C48015901EFEDFBE200814F
:106680001181228133810E945C3CA801B9018401FF
:1066900095010E94953DE0E6FCE200831183228390
:1066A00033838C019D010E94693C159507951595D2
:1066B000079515950795212F220F220B322F0E9447
:1066C0005C3C0E94B23E0E94693CA02F0B3008F057
:1066D000AAE00091B82B053C44F4063A34F0A83007
:1066E00010F4033B94F003E017C021EC35E20AE814
:1066F00018E20E94E5422AE838E213E501E03AD7C1
:1067000000EA10E035D700EB29C0A53010F40D3AAF
:1067100014F002E001C001E00093492CE0E6FCE245
:1067200000811181228133814091642C54E0459F86
:10673000F001E855F94D008311832283338328EC5F
:1067400035E20AE818E20E94E54200E510E010D7C1
:106750002AE838E213E501E00DD700E210E008D79F
:1067600023EF35E20AE818E20E94E5422AE838E21F
:1067700012E006E00E94930F0091492C10E01A935A
:106780000A930091B82B102F110F110B1A930A9333
:10679000B0E0BA93AA9328E036E20AE818E20E9431
:1067A000E54226962AE838E215E004E0E3D62DE13A
:1067B00036E20AE818E20E94E5422AE838E211E0EF
:1067C00001E0D8D694C00E94AC0DD0D68091BF2BEA
:1067D0009091C02B853E0CE0900714F084EE9CE075
:1067E0009A938A932CEC35E20AE818E20E94E5427B
:1067F00022962AE838E21AE003E0BCD600E310E073
:10680000B7D68D32914074F02EED35E20AE818E2E9
:106810000E94E5422AE838E215E007E00E94930F63
:1068200002E0A2D600E00093112C00933D2C0093CF
:106830003C2C2DC008E116EF95D60091480607FDC7
:1068400026C000E510E094D600E00E94B11810E2E6
:1068500000E384D600E61AEE85D68091BF2B909196
:10686000C02B853E0CE0900714F084EE9CE09A93D8
:106870008A932CEC35E20AE818E20E94E54222965F
:106880002AE838E21AE003E075D604E16DD60091FB
:10689000112C03950093112C043160F201E0009358
:1068A000312C75CE008107FD22C0E0E6FCE20081BC
:1068B0001181228133814091642C54E0459FF00185
:1068C000E855F94D008311832283338328E236E2B1
:1068D0000AE818E20E94E5422AE838E214E601E0FC
:1068E00049D600E210E044D600E510E041D6E8E4E5
:1068F000F6E0008106FFD6CF00E0E0E6FCE2008390
:1069000001830283038309E140CE0091372C0A956D
:106910000093372C19F40DE00093372C0091372C9D
:106920000093382C00913A2C013039F40091372C27
:106930000D3019F405E10093372C00E419D60091CD
:10694000372C0E94EB1E05E00FD628CD009148069B
:1069500006FD42C008ED16ED05D60091112C0395F9
:106960000093112C2091C92B3091CA2B10E02017D5
:10697000304060F700E6FCD50091282C0023A9F4F4
:1069800001E00093282CE4E2F6E000810D7F008313
:10699000E4E400810E7F008308EE1DEFE3D5009153
:1069A000272C10E00E94AB120CC000E00093282CB2
:1069B000E4E2F6E0008102600083E4E4008101602B
:1069C000008308E210E0D4D52091282C08EE11E0D5
:1069D000D3D502E0C9D58DCC0091372C0A95009310
:1069E000372C0E94EB1E00E410E0C2D504E0ACCFCF
:1069F00006E7402E01E0502E00EC602E02E0702EE3
:106A0000842D91E086159705A4F480932609909330
:106A1000270905E0A9D50E94C41A801691062CF416
:106A200048018093B62B9093B72B0A96861597054D
:106A300064F30091B62B1091B72B009326091093A5
:106A400027090E947C1D10E400E588D52091B72B12
:106A500001E010E091D52091B62B02E010E08CD53A
:106A600085D50091480606FD21C008EE1DEF7AD5B8
:106A70000091112C03950093112C2091C92B30917A
:106A8000CA2B2017304068F78824992401E000932E
:106A9000332C0E94631A0091642C002309F0A8CFC4
:106AA0000FE5402E01E0502E07E5A7CF0091332CD3
:106AB000002309F073CC0091372C0A950093372CF2
:106AC00000E410E055D53FCF27E436E20AE818E2AB
:106AD0000E94E5422AE838E21AE005E04BD500E8DA
:106AE00010E046D500E810E043D50AE03DD53ED59C
:106AF0000091480606FDDACF08EE1DEF33D5009170
:106B0000112C03950093112C2091C92B3091CA2B85
:106B10002017304068F72AD501E00093332C00E0BD
:106B20000093122C0093132C13D501E00093312C09
:106B30002DE236E20AE818E20E94E5422AE838E24D
:106B40001AE003E017D500E310E012D501E000934E
:106B5000312C0091C92B000F07D529E336E20AE852
:106B600018E20E94E5422AE838E21AE003E002D582
:106B700000E310E0FDD40091C92B000FF5D480E0B4
:106B800090E0A0E0E3EEFBE20081118122813381FD
:106B90000E945C3CA801622FB32EEFEDFBE2008166
:106BA0001181228133810E945C3C7B2DD3D4800FE4
:106BB000911F07E0D9D4A395AA3020F346EF5FEFE9
:106BC0008C010E94B33B0A5510400093122C109385
:106BD000132C093621E0120734F0E2E1FCE20856FA
:106BE0001140008311831091132C11233AF4E2E138
:106BF000FCE2008108591E4F00831183A9D401E0F3
:106C00000093312C0091C92BAFD4E3EEFBE200815D
:106C10001181228133810E945C3CA801622FB32E36
:106C2000EFEDFBE200811181228133810E945C3C07
:106C30007B2D90D4109F102D100D009F002D110D55
:106C4000212F220F220B322F0E945C3C0E94004316
:106C500040E050E060EB72E40E941E3E08F434CF46
:106C60002FE436E20AE818E20E94E5422AE838E218
:106C70001AE005E07FD405E210E07AD40AE074D48B
:106C800005E210E075D42091132C05E010E074D4D7
:106C90002091122C06E010E06FD42091152C07E013
:106CA00010E06AD42091142C08E010E065D41FCFC6
:106CB0000091480606FDFFCE08EE1DEF53D400916B
:106CC000112C03950093112C8091C92B9091CA2B04
:106CD000059610E08017904058F700E649D403E08D
:106CE0000E94B11810E200E339D440D402CB0091E5
:106CF000480606FD0FC008EE1DEF34D40091112C9C
:106D000003950093112C2091C92B3091CA2B201789
:106D1000304068F70091112C03950093112C2091BD
:106D2000C92B3091CA2B2017304008F064C0009165
:106D3000CB2B1091CC2B0E946E1E2091CD2B30912D
:106D4000CE2B0217130721F50E94191E2091CB2B81
:106D50003091CC2B02171307D9F424E536E20AE868
:106D600018E20E94E54205ECFBD300E210E000D4FB
:106D700000E510E0FDD32091CE2B0DEE11E0FCD309
:106D80002091CD2B0EEE11E0F7D327E302EF20C0C8
:106D90002EE536E20AE818E20E94E54200E8E0D378
:106DA0002FE636E20AE818E20E94E54200ECD8D36A
:106DB00000E011E0DDD300E211E0DAD300E411E0FD
:106DC000D7D303EF11E00E9455130395202F03EF53
:106DD00011E0D2D30091480606FFFCCF02EDC4D3E8
:106DE000E4E8F6E000810B7F008308ED04BF01E0DA
:106DF00000937900D3CA03EF11E00E9455130530C8
:106E000038F5E0912F2CF0E0EA5AF54D008103951A
:106E10000F70E0912F2CF0E0EA5AF54D008330918D
:106E2000622A330F330F330F330F1091632A312B44
:106E30000091642A10E1019F202D31290091652ADB
:106E400010E0202B2093CD2B3093CE2B0CE3A4CA43
:106E500020E836E20AE818E20E94E5422AE838E231
:106E60001AE003E087D30CE310E082D304E16CCD99
:106E7000008104FD22C210E010932A0810932B0811
:106E80000091372C0E3408F00BC2F2E00F9FF00196
:106E9000EE5DF64E05901490F001099400914806BD
:106EA00004FD33C000E61AEE5DD30091112C03956A
:106EB0000093112C8091C92B9091CA2B049610E05D
:106EC0008017904058F701E00093332C0091642C18
:106ED000002321F401E00093642C02C01093642C81
:106EE0003BD32091642C04EF11E046D300E510E081
:106EF0003FD306E410E03CD302E0C02EDD2401E0E5
:106F00000093312C08E030D34CCA0091332C00237D
:106F100009F0C6C10091292C073011F489E001C0A5
:106F200086E00091412C03950093412C082F10918D
:106F3000412C011710F48093412C2091412C03E047
:106F400010E00E94D813ACC10091462C0395009329
:106F5000462C0D3018F00CE00093462C0091462C86
:106F60000093472C2091462C06EF11E005D398C1E1
:106F70000091352C03950093352C043018F003E074
:106F80000093352C2091352C08EFEFCF00914A2C3F
:106F9000039500934A2C053018F004E000934A2C26
:106FA00020914A2C07EFE1CF00914B2C03950093E1
:106FB0004B2C053128F004E100934B2C00E5D8D28E
:106FC00020914B2C06E4029F80010E94D81720914B
:106FD0004B2C0CE010E0D0D205E0C6D20E94C41ABF
:106FE0000093262C5DC10091402C03950093402C0A
:106FF000053018F004E00093402C0091402C0E94D2
:10700000681D2091402C04E110E0B0CF00913E2C8F
:10701000039500933E2C0B3018F00AE000933E2CB1
:1070200020913E2C0BE1A2CF00913F2C03950093C1
:107030003F2C083018F007E000933F2C20913F2CA4
:107040000DEF11E099D288D22BC10091422C0A9504
:107050000093422C0F3F11F41093422C2091422CAC
:107060000CE184CF0091432C03950093432C0A300C
:1070700018F009E00093432C08EE13E00093660932
:10708000109367092091432C04E6029F00926A093D
:1070900010926B090E94FE1F2091432C09EF65CFCF
:1070A0000091242C03950093242C04301CF003E061
:1070B0000093242C2091242C0BEF57CF00912A2CE5
:1070C000039500932A2C0B3518F00AE500932A2C1F
:1070D00020912A2C09E14ACF00912B2C0395009393
:1070E0002B2C0F3118F00EE100932B2C20912B2C20
:1070F00002E13CCF0091282C013009F0D1C0009171
:10710000272C03950093272C063618F005E60093EC
:10711000272C0091272C0E94AB122091272C09EEDE
:1071200024CF0091652C03950093652C043018F052
:1071300003E00093652C10D22091652C0AEF15CF47
:107140000091442C0A950093442C0A3018F40AE06C
:107150000093442C2091442C0CEF11E00DD200E35D
:1071600015E700D29DC00091642C03950093642C18
:10717000023018F001E00093642CEED12091642CD1
:1071800004EFF3CE0091642C002311F48FE501C0CD
:1071900086E791E0E6EBFBE20081118101501040AF
:1071A000008311830817114014F4808391830091A8
:1071B000B62B1091B72B00932609109327090E9434
:1071C0007C1D2091B72B01E010E0D6D12091B62B89
:1071D00002E01ACFE2E1FCE2008111810F5F1F4F54
:1071E00000831183083611401CF000E00083018306
:1071F000AFD12091132C05E010E0BED12091122CCC
:1072000006E010E0B9D12091152C07E010E0B4D1D0
:107210002091142C08E0F8CE0091480605FD40C0EE
:1072200000E00093182C0093192C0093162C009367
:10723000172C04E69DD10E94BA192091182C309188
:10724000192C0091162C1091172C0E94431806E05F
:1072500026C000912C2C039500932C2C023019F49D
:1072600001E000932C2C20912C2C0FEF11E084D105
:107270007DD116C002E000933A2C0DE40093372C28
:1072800002E376D1F5CF00912F2C039500932F2C9C
:10729000003118F00FE000932F2C68D104E064D186
:1072A0000091532C002319F408E210E061D104E0AE
:1072B0005BD101E00093312C71C8008105FD6EC8DF
:1072C00000E010E000932A0800932B080091372C6F
:1072D0000E3430F7F2E00F9FF001E254F64E0590C5
:1072E0001490F00109940091480605FD2AC000E5BC
:1072F00013EC38D10091112C03950093112C80913F
:10730000C92B9091CA2B089610E08017904058F72F
:1073100001E00093332C0091492C03950093492CF4
:10732000043018F001E00093492C2091492C0DE025
:107330000E94D81308E210E01BD102E0C02EDD2429
:1073400030C80091332C002309F0AACF0091412CC2
:107350000A950093412C09F0F0CD01E00093412CF7
:10736000ECCD0091462C0A950093462C0F3F09F076
:10737000F5CD1093462CF2CD0091352C0A95009353
:10738000352C0F3F09F0FECD1093352CFBCD00912D
:107390004A2C0A9500934A2C09F002CE01E0FECD5A
:1073A00000914B2C0A9500934B2C0F3F11F4109336
:1073B0004B2C20914B2C06E4029F80010E94D81791
:1073C00020914B2C0CE010E0D7D006E006CE0091C7
:1073D000402C0A950093402C09F00FCE01E00BCE13
:1073E00000913E2C0A9500933E2C033008F018CEF5
:1073F00003E014CE00913F2C0A9500933F2C0F3FE1
:1074000009F01CCE10933F2C19CE0091422C03950D
:107410000093422C0A3008F421CE09E00093422C5C
:107420001DCE0091432C0A950093432C0F3F09F089
:1074300023CE1093432C20CE0091242C0A95009348
:10744000242C01300CF036CE01E032CE00912A2CF3
:107450000A9500932A2C003508F03ACE00E536CE86
:1074600000912B2C0A9500932B2C0F3F09F03ECE58
:1074700010932B2C3BCE0091282C013009F010CF1B
:107480000091272C0A950093272C093508F041CE4E
:1074900009E53DCE0091652C0A950093652C0F3FC0
:1074A00009F049CE1093652C46CE0091442C0395EB
:1074B0000093442C013508F44DCE00E549CE0091EF
:1074C000642C0A950093642C0F3F09F056CE10935C
:1074D000642C53CE0091642C002311F487E501C085
:1074E00080EC92E0E6EBFBE2008111810F5F1F4F21
:1074F00000831183801791070CF059CE56CEE2E13C
:10750000FCE20081118101501040008311830AF0D8
:107510006FCE08E611E0008311836ACE0091480621
:1075200004FDBECE7DCE00912C2C0A9500932C2C10
:107530000F3F09F098CE10932C2C95CE00912F2C54
:107540000A9500932F2C0C3008F0A7CE0CE0A3CEA8
:107550000C94151B0C94741A0C94E71D0C94571A78
:107560000C94C0100C946A200C945F200C944C0E68
:107570000C94371A0C94340F0C94951300008895D2
:10758000FECF11231AF4119501951040980189013D
:1075900008950E94943EC801D9012A013B015CD0A4
:1075A00057D071F48201930153D051F401E2EEE619
:1075B000FCE2008341830FEF1FEF2FE73FE73DC061
:1075C00044D0A201B3010E94BB3CAC01BD0140D03C
:1075D00061F442D03AD00E94363E0BED1FE029EC18
:1075E00010F43FE32AC03FEB28C0A201B3012DD025
:1075F0000E94953D080119012FD0820193010E943C
:107600001E3E23D0A0F41CD050F424D0A801B90110
:107610000BED1FE029E430E40E94FF3C0EC01AD0BD
:107620004BED5FE069E470EC0E94BB3C06C008D003
:1076300010F410D002C00ED03058E8E00C94A53EF3
:107640000E94363E8001910108958C019D010895AC
:107650000C94143E0C94964140E050E060E070E0E1
:1076600008953F7741E00C94354203E20DBF01E2FB
:107670000EBFC0E0D1E20E94353F002311F00E940E
:1076800018420E947A200E94BE3A0C94BE3A0D0124
:10769000DA0140E050E060E070E00E94143E39F40E
:1076A00000E010E04D934C9320E030E00CC0B901B5
:1076B000660F771F7E57572F550F550B7D935C93A1
:1076C0002F7730783F63D00108954A9512F0000F6C
:1076D000E1F708954A9512F00695E1F70895002420
:1076E000E8E0EA9532F0001F001C0416D0F3041AFB
:1076F000F8CF001F402D00950895FF27442312F472
:10770000F1604195002312F4F09501950E946F3BC2
:10771000F0FD0195F1FD41950895149F102D059FF1
:10772000100D049F002D110D08954A951AF015951E
:107730000795FBCF089500241124EFE0001F111FCF
:10774000001C111C0416150610F0041A150AEA95FF
:10775000AAF7001F111FA0010095109508955195DB
:10776000419550400895FF27552312F4F160F7DF4B
:10777000112312F4F09507D00E949B3BF0FD03D03B
:10778000F1FDEDCF089511950195104008954A95AA
:107790002AF03695279517950795F9CF08954A95BC
:1077A0002AF03595279517950795F9CF0895002468
:1077B00011241001E0E2EA9592F0001F111F221F30
:1077C000331F001C111C221C331C04161506260630
:1077D000370688F3041A150A260A370AECCF001F69
:1077E000111F221F331FA001B10100951095209594
:1077F00030950895FF27772312F4F16015D03323D5
:1078000012F4F09509D00E94D73BF69508F404D005
:10781000F69508F409C008953095209510950195C6
:107820001F4F2F4F3F4F089570956095509541958C
:107830005F4F6F4F7F4F0895FF27112477FB660F2F
:10784000771F089409F4771F679517F8EE2700242F
:1078500037FB220F331F089409F4331F279507F8CD
:10786000089527FD0EC0EE0F001F111F221F3A952D
:107870003230B8F7332319F427FD31E002C027FF77
:1078800030E0E03821F400FF08940EF488940F4FA4
:107890001F4F2F4F3F4F323038F4332319F427FD59
:1078A00031E002C027FF30E03F3F29F0220F000CFB
:1078B000379527950895ACC0032E002012F40E943E
:1078C0000C3CE02F012F122F232F3EE9D1CF0024B3
:1078D000F8CFBCDF432F4F5748F04F3148F007FC3B
:1078E00091C03FE72FEF1FEF0FEF089533278CC0B4
:1078F000322F212F102F0E2F4F5141950E94C73B41
:1079000007FE08950C940C3CF901EE0FFF1F37FBA6
:10791000FF3F31F0EF2BE12BE02B8894B8940895D2
:10792000E02BE12B21F008949894B8940895989452
:10793000889438940895FB01EE0FFF1F77FBFF3FFB
:1079400031F0EF2BE52BE42B8894B8940895E42BC9
:10795000E52B69F3E8CFEFDF68F021F43723262F1A
:107960008A010895372FFBCFE6DF20F00BF0089552
:107970007327EAF751C0C8DFE8F3B3F361F3DBDF45
:10798000C8F383F3A1F358DF401751076207730769
:1079900031F4011411F10024E89488942BC078F09C
:1079A000332E372F732D322E262F632D312E152F88
:1079B000532D302E042F432D302C012C132C371730
:1079C00039F0669557954795F795E0407395F7CF51
:1079D000E7FBEE0FE0E010246AF0EF0F041F151F25
:1079E000261F60F4279517950795E79508F4689486
:1079F00033953ECFEF0B040B150B260B39CFE0E888
:107A00007E27B9CF302D30782227112700270895FF
:107A10003FE7302920E8F9CF3FEF2FEFF6CF8BDF9C
:107A2000D8F3D1F370783727089585DFA8F3A3F34F
:107A3000F9CF3078372793CF67DF70F383F3A9F35B
:107A40007ADF50F3B3F3A9F3F7DE0124E8943F574C
:107A5000E040370FEF1F12F0D9F603C03A3E90F224
:107A60006894E0E00A92AA933A93AA273324222446
:107A70003327049FF001059FF00D712D731F149F94
:107A8000F00D711D221C069F700D211C331C159FCB
:107A9000700D211C331E249F700D211C331E169F58
:107AA000200C311CAA1F259F200C311CA31F269FD0
:107AB000300CA11D39915EF43395A6953794279427
:107AC0007795F795E79533953130BCF316C0AA2327
:107AD00022F0332351F4339510C0339571F4A991FA
:107AE000099096CFA7FD09C03A95EE0FFF1F771FAB
:107AF000221C331CAA1F3230A8F7E894FE2B09F091
:107B000068942A2F8101E72FA9910990BACE13DF3B
:107B100010F00BF087CF80CF0EDFE9F3E0F3032EF8
:107B2000072670CF032E072673CFEEDEA0F37BF37C
:107B300099F301DF80F39BF3A9F37EDE012427FD97
:107B400006C0000F111F221F3150E040F8CF67FD23
:107B500006C0440F551F661F7150F040F8CFE894DF
:107B6000371BEF0B3158EF4F2AF0EE23E9F63F3F7A
:107B7000D9F203C03A3EA8F26894E0E0F0E01124A4
:107B8000139440175107620738F0315008F4689495
:107B9000000F111F221FEE1F041B150B260BEF0BEE
:107BA000000F111F221FEE1F0A9279E17A95AAF0A9
:107BB000041715072607EF0730F0041B150B260BDB
:107BC000EF0B089401C08894111C221C331C001C6C
:107BD000000F111F221FEE1FE9CFF0F9E894E22BEE
:107BE000E12BE02B09F068940694379427941794BE
:107BF000E79508F468947395B9F30990332311F06D
:107C0000F0FF09C0369427941794E79508F4689418
:107C100033953130BCF3012D122D232D32CE8BCE76
:107C200098940895189408956FDED0F3C1F383DE1D
:107C3000B8F3041715072607370708957CDEA0F070
:107C400063DE90F029F0E32FE7273AF473170895E5
:107C500072DE51F04EF008940895041715072607B8
:107C6000370719F016F4B8F78894089564DEE0F346
:107C70004BDED0F3E7DFC0F308940895759165916A
:107C800055914591159011FA259035900895F9DF99
:107C9000041B10E003C0F4DF041B150B20E030E0F0
:107CA00005C0ECDF041B150B260B370BB8F010FCDE
:107CB00017C045910590E00FF11F0417100540E033
:107CC0002407340758F436F404910024F101E01B32
:107CD000F0090994E00FF11F25903590F101099406
:107CE00011F4D6F7F1CF31960EF0319650E060E006
:107CF00070E045914B3F48F089F34F3F29F04E3FEC
:107D000011F07591659155914591041B150B260B4A
:107D1000370B39F318F3E7CFFA92EA92DA92CA9264
:107D2000BA92AA929A928A927A926A925A924A92B3
:107D3000BA93AA939A938A930895FF84EE84DD847C
:107D4000CC84BB84AA84998488847F806E805D8083
:107D50004C80BB81AA8199818881F0E0EC0FFD1FE6
:107D6000EF0108950E94903E229741E050E060E0CC
:107D700070E00E941E3E60F440E00E94143E21F438
:107D800002E26BD03FEF5FC001E267D03FE75BC02C
:107D9000AE010E94473BC801D90143EF54E065E3BF
:107DA0007FE30E941E3E68F437FBAA0FBB1FB3950A
:107DB000B695A795B7F9088119810150104008833D
:107DC000198340E050E060E87FEB43D0280139019F
:107DD00040E050E060E87FE33CD0A801B9018201B7
:107DE00093010E94953DC801D901A801B9012FD086
:107DF000280139010881102F110F110B212F312F6C
:107E00000E945C3C48E152E761E37FE320D04801F7
:107E1000590142E252E964ED7EE38201930117D0F9
:107E20004DED5BE96AE27FE316D0A201B3010FD00A
:107E300044E050E060E070E40ED0AC01BD0107D03A
:107E4000A401B50108D02296ECE00C94A13E0C945C
:107E50001C3D8C019D010C94BB3CEEE6FCE20083D2
:107E600051830FEF1FEF2FE7089501E008950E945F
:107E70008C3EEF97EF976A972A873B874887598709
:107E800068017B0100E00B830C8302C011D21BD27E
:107E90000AD2053251F00023C9F70B811C81EF96FD
:107EA000EF966A96E0E10C949D3E0081053221F444
:107EB00002D2FED105E2EBCF00E00F830E830A83EE
:107EC00009833E0102E1600E00E0701E02EB16E243
:107ED000088B198B06C00981002311F400810983E6
:107EE000EAD1D9D10052B9F3035059F00850B1F397
:107EF000025019F0035049F00CC00A8103950A831F
:107F0000EFCF0E8103950E83EBCF0F8103950F8387
:107F1000E7CF00810A3279F4AAD1AD90BD9098D113
:107F2000BB203AF4B194A19400E0B00A0A81039511
:107F30000A83C1D114C0AA24BB244AE050E00DC07A
:107F400021916F0185010E948D3BA22EBB24A00EC2
:107F5000B11E00EDA00E0FEFB01EA0D188F30A8174
:107F6000002311F000E00F8396D10E32F1F4A3D17B
:107F700092D10A3231F47BD18D909D9069D19BD101
:107F800017C0882499244AE050E088D188F42191D0
:107F90006F0184010E948D3B822E9924800E911ED8
:107FA00000ED800E0FEF901EF0CF88248A94982C5D
:107FB00080E071D10C5421F00C5131F0045039F4AF
:107FC00081E0C80E7AD103C001E0C00ED81E6BD18B
:107FD000EAE5FAE10C94473E80FB5EF44B815C815C
:107FE000652F660F660B47D140835183628363839D
:107FF0004FCF2B813C813FD12083318349CF37D173
:108000000D91119625D10A8B2E0103E115D1E0C007
:108010002ED16D907D901CD1062D072921F403EC03
:10802000602E06E2702E992022F400E1802E07E2F5
:10803000902E80E090E001C00196F30101913F0194
:10804000002319F088159905BCF30CD123019195F3
:1080500081959040680E791EBBC00E81002331F0DF
:10806000082D092919F499248824839402ED16E235
:10807000088B198B0881003739F4F9D0ECD000E176
:10808000D5D000E0098330C0F1D046F40D911D91A8
:108090002D913D91DDD0C801D90101C0DCD008810E
:1080A0000F3611F408E0ECCF053749F70AE0E8CFC6
:1080B000DDD04D915D9126F46D917D91C9D005C0C3
:1080C000C7D0652F660F660B762FCA01DB017723B9
:1080D0004AF40DE209839095A095B09581959F4F44
:1080E000AF4FBF4F0AE0A2D03E0107E9600E00E0AB
:1080F000701E2E0107E9A0D0082F092B0A2B0B2B8D
:1081000011F001E001C000E00D83082D092919F4E8
:108110000D8100FF1FC094D0E889F989E00DF11DA1
:108120000081F30102933F018BD0C801D901012BDB
:10813000022B032B81F799206AF40F81002351F061
:10814000A3D010E04501801A910A04C000E3F301B6
:1081500002933F018E0109561F4F06191709081592
:108160001905A4F30E81002399F10D8100FF30C0A1
:108170000881083711F0083549F474D0F3010881FB
:10818000008370D000E3F301008322C00F3601F5B5
:10819000F30100810033E1F000E302933F0118C0D6
:1081A00003EE602E06E2702E462C502EF201008166
:1081B000002371F001E040D0F9CF0FEFC00ED01EC8
:1081C00006E0602E07E2702E09E0402E07E2502EF6
:1081D000420186189708A814B9041CF480E090E0C6
:1081E00007C052D0A818B90810E0A01AB10AC501FA
:1081F0000A81002321F401C063D00197EAF70981C5
:10820000002339F055D004C053D0F30101913F0150
:108210005AD00FEF800E901EBAF70A81002309F49E
:1082200037CE01970AF434CE4BD0FBCF10E00C8749
:108230001D871E871F870895400E00E0501E089579
:108240004C855D856E857F858C019D010C94D73BA7
:10825000A083B18308958D919D91A083B183A0E007
:10826000B0E008950FEF600E701E089580FBF701D7
:10827000A081B1810895F701A081B1810D911D9177
:10828000A083B183F80108950981002311F001E072
:10829000089500E00895F60100810895F601008137
:1082A00000530A300895F60101916F010883089583
:1082B00028853985089501E0C00E00E0D01E08959C
:1082C0002885398500E2EA85FB8509950B811C81AB
:1082D0000F5F1F4F0B831C8308950E94983EC801B7
:1082E000D9011A013F7740E856E968E17BE40E9432
:1082F000363E38F416D0B38300E010E020E030E0E2
:108300000DC03B2F0E94693C0E945C3C0AD0338325
:10831000A801B9018C019D010E94FF3CE4E00C948E
:10832000A93EF10100831183228308950E948C3EAF
:10833000C801D901BF7741E050E060E87FE33B2FFF
:108340000E941E3E70F440E00E94143E29F40BEDA2
:108350001FE029E43FE350C0CC24DD24EE24FF24B9
:108360001CC00BEDC02E0FE0D02E09E4E02EF72E3E
:1083700040E07FEB082F48D02801390140E050E071
:1083800060E87FE38C019D013FD0A801B901820123
:1083900093010E94953DC801D901AC01BD018C013A
:1083A0009D012DD02801390144E25FEF6BE27CEBA7
:1083B00026D048E854E466EA7EE328D048E150EC51
:1083C0006FE370E423D045EB1CD0480159014AEE1D
:1083D00054EB66E870E48201930118D046EB11D0AB
:1083E000A801B901840195010E94953DAC01BD0130
:1083F00006D0A601B70108D0E0E10C949D3E0C9494
:108400001C3D5DEF68E670E40C94BB3CFDDFA2010F
:10841000B301F5CF20E006D0E9F70895259102D009
:10842000E9F708952D9301501040202F212B089536
:108430008AEE96E8FC0105911491FC013296A59113
:10844000B491FC01349625913491422F432B19F0BD
:10845000F901E4DF01C0DEDF069616E8863F9107EA
:1084600048F3089540E00C9435420E94943E2897CA
:10847000802FB32F442E40E050E060E070E00E9477
:108480001E3E10F401E001C000E0000F400EBF7777
:1084900043E859EF62E27FE3082F3B2F80D076D08C
:1084A00041E05CEF6FE777E40E94363E88F5AE016D
:1084B0000E946D416BD0042D10E06BD04881598132
:1084C0006A817B8172D0088319832A833B83AE0142
:1084D0004C5F5F4F2A0140E050E060E87EE35FD0F0
:1084E000A2010E946D4140E050E060E870E40C8120
:1084F0001D812E813F8153D0A801B90108811981C6
:108500002A813B810E94FF3C0E94693C402E0CC0A6
:108510000E94693C602E3DD0A801B9018C019D01EB
:1085200033D0460C03E0402240FA3EF4AC01BD01DA
:1085300000E010E020E83FE327D002E0401608F01A
:10854000B0588C019D0129D0280139014BEF57ED1E
:108550006EE179E324D045E656E269E97BEB21D070
:1085600048E554E363EA7DE31CD041EE5DE565E256
:108570007FEB17D04BED5FE069EC7FE316D00DD0B9
:108580002896E8E00C94A53E0E94FF3CC801D90162
:10859000089520E030E00C94673CAC01BD010C94E0
:1085A0001C3D03D0A201B301FACF0C94BB3C1B2F9E
:1085B0006A2FF901A081B181AD014F5F5F4F408308
:1085C00051830C93A62FB12F0895BA93AA932497A1
:1085D0000A831B8389019E012A5F3F4F28833983C9
:1085E000BE01AE014E5F5F4F27ED32E40E94373F80
:1085F00020E0AA81BB812C932496A991B99108957A
:108600000E94903E22974801590141E050E060E00D
:1086100070E00E941E3E98F440E00E94143E29F44F
:1086200000E010E020E030E04EC001E2EEE6FCE2C7
:10863000008351830FEF1FEF2FE73FE744C0AE01E8
:108640000E94473BC801D90145EC53E062E47FE357
:108650000E94BB3C4AE151E562E17FE33BD0A801C7
:10866000B9018C019D013BD0402E088100FF14C050
:108670000A952DD0802F43EF54E065EB7FE3042D66
:108680000E941C3D37FB220F331F380F369527956C
:1086900037F9C801D9010BC01AD0842D912FD90107
:1086A00037FBAA0FBB1FB00FB695A795B7F940E0EF
:1086B00050E060E87EE38C019D010CD0AC01BD016F
:1086C000840195010CD02296ECE00C94A13E42E08E
:1086D0000C947D3B0E941C3D2801390108950E94A5
:1086E000953DA201B3010C94BB3CE6052421F6861E
:1086F00066050A27000050524F46494C4500CFD02E
:10870000CED4C8CBDC004241545445525900C1C0BC
:10871000D2C0D0C5DF004652455155454E435900A1
:10872000D7C0D1D2CED2C000465245512E00D7C0BC
:10873000D1D2004645525249544500D4C5D0D0C884
:10874000D200434F494C20424C2E00C1C0CBC0CD7B
:10875000D100454E472F505943005059432F454EA5
:108760004700564F4C554D452020202000C3D0CE09
:10877000CCCACED1D2DCFAFA004154414B20564F3C
:108780004C2000C0D2C0CAC0FAC3D0CECCFA00542C
:108790004F4E4520564F4C202000D2CECDFAC7C2B6
:1087A000D3CAC0FAFAFA00504F574552202000D2DF
:1087B000CECAFAFAFA004741494E20202020202054
:1087C0002000D3D1C8CBC5CDC8C5FAFA0046494C64
:1087D000544552202020202000D4C8CBDCD2D0FA2F
:1087E000FAFAFAFA00444953432D2000C4C8D1CA0A
:1087F000FC0053454E532046452020202000D7D36F
:10880000C2D1D2FAC6C5CBFAFA004C454420425236
:1088100049474854202000DFD0CACED1D2DCFAFA32
:10882000FAFA00444953504C45592020202000DDDD
:10883000CAD0C0CDFAFAFAFAFA00484F542053547D
:108840004F4E45202000C3CED0FACAC0CCCDC8FAC6
:10885000FA0054524553484F4C44202000CFCED00C
:10886000CEC3FAFAFAFAFAFA00414C4C204D4554BC
:10887000414C2000C2D1C5FACCC5D2C0CBDB002010
:108880004E4F2049524F4E2000C1C5C7FAC6C5CB36
:10889000C5C7C00020204649454C4420202000FA8E
:1088A000FAFACFCECBC5FAFAFAFA002020424541B7
:1088B0004348202000FAFAFACFCBDFC6FAFAFA00D2
:1088C00020536561424541434800CCCED0D1CAFA1D
:1088D000CFCBDFC6FA002052554242495348200010
:1088E000FAFAFACCD3D1CED0FAFA00202050415275
:1088F0004B20202000FAFAFACFC0D0CAFAFAFA00C8
:108900002043752B41672B202A00CCC5C4DCFAEF2D
:10891000EBFEF10044656D6F004F4646004F4E0080
:108920002D253032642D200020504C4541534520E8
:10893000574149540020202020212053204F20530C
:108940002021003C4F46463E0020204C6F772042BD
:108950006174746572792021002045524153494E5B
:108960004720454550524F4D004B504F542D004B22
:108970000050004F00540050524F32200025730029
:10898000464D202D202564206D487A200020476C1C
:108990004F42414C204552524F522100256C6400F9
:1089A000203D2020442045204D204F20203D006DBB
:1089B00061696C3A20726164696F646F6D40692E01
:1089C0007561002020202A20253032643A2530327B
:1089D0006420202A00466163746F72792073657485
:1089E00074696E677300204B657920656E747279C7
:1089F0002000256420487A202A203C303E0025644F
:108A0000206D41202A203C2D3E203C2B3E0025306D
:108A100034642E006D5620002020205475726E2084
:108A2000636F696C21002530326425632530326420
:108A300000436F696C2E422000202020202020005F
:108A400047256420532564204625642563256476E4
:108A5000256400502564282564292564487A20006F
:108A6000253032640025303264200050494E0052D7
:108A7000002D202564200028256429202D20256430
:108A8000202020002D202564202000464D2020207D
:108A900020202D2025646D487A2000284F46462945
:108AA00000284F4E29200020003E002D2025640084
:108AB0002D2025642E2564205600282564292D208C
:108AC0002564487A20002D2025642067722020002C
:108AD000282573292D2564206D56202020004B4524
:108AE00059204F4B2120202000456E747279204B75
:108AF00045592020202D2C2B20006F002020204BBA
:108B0000455920204F4B2021212000762E20303146
:108B10002F30382F3232004B65793A2025582825DE
:108B2000642D25642900253032643A2530326420D2
:108B3000436F64655F002558255800456E742E4BC1
:108B400065793C25643E202530345820003C562E63
:108B500050323E006D61696C3A20726164696F64E5
:108B60006F6D40692E7561202000687474703A2022
:108B7000726164696F646F6D2E6F7267002A2044A2
:108B8000454D4F202A004572726F722043552B4E7F
:108B9000692B004572726F7221004F4B20002A2A08
:108BA0002A202564206D56202A2A2A2020202000F1
:108BB000436F696C20626C2E707265737320274D51
:108BC000656E752700416D706C69742E2050686168
:108BD00073652046696C746572003C253032643ED2
:108BE000203C253032643E203C4625643E20004730
:108BF0007261756E6420626C2D002D4F4B2D00202C
:108C00004E6F2046657272697465002054616B6511
:108C1000204665727269746500204572726F722118
:108C200000204F4B2100204F4B21202020202000EE
:108C300020726164696F646F6D40692E75612020D8
:108C40000020202020204552524F52212020202059
:108C500020002020204552524F52203E3D352021F9
:108C6000202020003C204F4646203E000080C0E0EF
:108C7000F0F8FCFE00921E7900010AD723BD0AD746
:108C800023BD400130313233343536373839414233
:108C90004344454600286E756C6C20706F696E7495
:108CA00065722900303132333435363738396162F4
:108CB0006364656600464C4F4154533F2077726FA2
:108CC0006E6720666F726D617474657220696E7371
:0C8CD00074616C6C656421003F3F3F0044
:0400000300000000F9
:00000001FF
